:1000000056C6000073C6000071C600006FC600002F
:100010006DC600006BC6000069C6000067C6000020
:1000200065C600000C94D01A61C600000C94801ABA
:100030005EC600005BC600000C94A81A57C60000FC
:100040000C94581A53C6000051C600004FC6000059
:100050004DC600000C94FF1A49C6000047C60000B8
:1000600045C6000043C6000041C600003FC6000070
:100070003DC600003BC6000039C6000037C6000080
:1000800035C6000033C6000031C600000E12101243
:100090001012131213121312131213121612181233
:1000A000181218121812301234126B21E6219E20F9
:1000B000EC1FAC23CC219E22DA22FE22CE24F42691
:1000C000D327EC274628D42A4D2981298B29A42916
:1000D000C129942AA32AD42ADA2AF12B172C5526CF
:1000E00074266D266D2658265B265E266D266D26A7
:1000F0006D266D26612664266D2667266A26DF2C0E
:10010000432D652C4E2CF52E402DCA2ECE2EE22EE0
:10011000A3309C2F8430C030CF318E3295323E34A4
:10012000E732EA3245333E3454337F33B4339333CA
:10013000172F202F272F2E2F352F492F572F632F83
:100140006D2F4635FB344835483548351035483530
:1001500048353335483546354635483548354835D0
:10016000483548354835483548354835EB34F3345B
:100170002F5341564553001F1C1F1E1F1E1F1F1EBD
:100180001F1E1F10278813D007E803E803E803F4B5
:1001900001F401320032003200320081008000425E
:1001A000415700544150002E424157002E574156AE
:1001B000002E54415000EFEEE6E0EBF3E9F1F2E0FF
:1001C0002E2E00776169742E2E2E00CFEEE4EEE61F
:1001D000E4E8F2E500506C656173650020EEF8E834
:1001E000E1EEEA00206572726F727300D2E0E9EC12
:1001F000E0F3F220E7E0EFE8F1E800577269746598
:100200002074696D656F757400D2E0E9ECE0F3F27B
:1002100020F7F2E5EDE8FF00526561642074696D36
:10022000656F757400D2E0E9ECE0F3F220522F57CD
:1002300000522F572074696D656F757400C7E0E335
:10024000F0F3E7EAE000506C6179696E6700D1CEA7
:10025000D5D0C0CDC8D2DC20CAC0CA005341564553
:1002600020415300EAE0F0F2F320EFE0ECFFF2E887
:100270000053442D4341524400C2F1F2E0E2FCF24B
:10028000E500496E7365727400F4E0E9EBE0006626
:100290006F726D617400CDE5E2E5F0EDFBE920F4ED
:1002A000EEF0ECE0F20057726F6E672066696C65E5
:1002B00000F4E0E9EB0066696C6500CDE520ECEE4A
:1002C000E3F320F1EEF5F0E0EDE8F2FC0043616EBF
:1002D000277420777269746500F4E0E9EB006669C1
:1002E0006C6500CDE520ECEEE3F320EFF0EEF7E8EF
:1002F000F2E0F2FC0043616E2774207265616400D5
:10030000F4E0E9EB0066696C6500CDE520ECEEE316
:10031000F320F1EEE7E4E0F2FC0043616E27742085
:1003200063726561746500CED8C8C1CAC000455209
:10033000524F5200CAEEEDF2F0E0F1F2EDEEF1F2C2
:10034000FC00436F6E747261737400C7E0ECE5EDFE
:10035000E8F2FC20E5E3EE3F005265706C616365F6
:100360002069743F00D3E6E520F1F3F9E5F1F2E20C
:10037000F3E5F200416C7265616479206578697318
:10038000747300D1E5EAF2EEF03A2000536563742D
:100390006F723A2000CAEBE0F1F2E5F03A20004338
:1003A0006C75737465723A2000D0E0E7ECE5F0FB01
:1003B0000053697A657300D0E0E7E4E5EB00506133
:1003C00072746974696F6E3A00455854454E4445DD
:1003D00044204C4241004641543136204C424100B9
:1003E0004641543332204C4241004641543332009E
:1003F000464154313600457874656E646564004644
:1004000041543136202833324D622900464154315F
:10041000320046726565002000290028002F004B3D
:1004200000CCE1004D4200CDE5E8E7E2E5F1F2E580
:10043000ED00556E6B6E6F776E00D3EDE8E2E5F080
:10044000F1E0EBFCEDFBE900556E697665727361D6
:100450006C005375706572466C6F707079004861FE
:1004600072644469736B20284D42522900D4EEF027
:10047000ECE0F23A00466F726D61743A00D0E5E24A
:10048000E8E7E8FF3A20005265766973696F6E3AD3
:100490002000C8ECFF20EFF0EEE4F3EAF2E03A00CF
:1004A00050726F64756374206E616D653A00CEE1C1
:1004B000FAE5EC0053697A6500D1E5F02E20EDEE07
:1004C000ECE5F00053657269616C206E756D6265D4
:1004D0007200CFF0EEE8E7E2EEE4E8F2E5EBFC00D4
:1004E0004D616E75666163747572657200D1E2EE7E
:1004F000E1EEE4EDEE2C20CCE100467265652C20A7
:100500004D4200C1EBEEEAE83A00426C6F636B7358
:100510003A00E1E0E9F200627974657300E100629B
:1005200000EFE8EBEEF20070696C6F74007777779C
:100530002E74726F6C736F66742E72750032303168
:10054000352D323031360085864F6C656720547208
:1005500069666F6E6F7600762E20312E312E310057
:100560005A5820546170657200F1E8E3EDE0EBE069
:100570002E2E2E00746865207369676E616C2E2EB6
:1005800000CEE6E8E4E0EDE8E50057616974696EE5
:100590006720666F7200EDE0F1F2F0EEE9EAE83F05
:1005A00000746F2064656661756C743F00D1E1F082
:1005B000EEF1E8F2FC0052657365742073657474A3
:1005C000696E677300CFEE20F3ECEEEBF7E0EDE839
:1005D000FE0044656661756C7400CEEFF0E5E4E5FD
:1005E000EBE8F2FC0044657465637400C7E0F5E273
:1005F000E0F2004361707475726500C4E0EDEDFBDC
:10060000E5004461746100D1E8EDF52E32005379C4
:100610006E63203200D1E8EDF52E310053796E6320
:10062000203100CFE8EBEEF20050696C6F7400CF20
:10063000E8EBEEF22EE40050696C6F742E6C00EC67
:10064000EAF100757300ECF1006D7300F4F0EEED6B
:10065000F2007269736500F1EFE0E40066616C6CB2
:1006600000D0F3F10052757300C0EDE300456E67F2
:1006700000783800783400783200783100C0E2F237
:10068000EE004175746F00C2FBEA004F666600C25F
:10069000EAEB004F6E00CAEEEDF2F0E0F1F200D1AD
:1006A0006F6E747261737400C4E0F2E020E820E2BF
:1006B000F0E5ECFF004461746520262074696D65E7
:1006C00000D2E0E9ECE8EDE3E80054696D696E679B
:1006D0007300D1EAEEF0EEF1F2FC00537065656450
:1006E00000CFEEE4F1E2E5F2EAE000486967686C09
:1006F0006967687400C7E2F3EA20E7E0EF2E005371
:100700006F756E642072656300C7E2F3EA20E2F160
:10071000EFF02E00536F756E6420706C617900C726
:10072000E2F3EA20EAEBE0E22E00536F756E6420FC
:100730006B657900DFE7FBEA004C616E6775616706
:100740006500C8CDD4CE0041424F555400534420DB
:10075000CAC0D0D2C000534420494E464F00CDC03D
:10076000D1D2D0CEC9CAC80053455454494E47537C
:1007700000D1CED5D0C0CDC8D2DC00534156450003
:10078000CFD0CED7C8D2C0D2DC00504C415900C720
:10079000E0E3F0F3E7EAE02E2E2E004C6F6164698F
:1007A0006E672E2E2E00C3EEF2EEE2EE00446F6E68
:1007B00065003CCFF3F1F2EE3E003C456D7074797C
:1007C0003E00CEF8E8E1EAE02043524300435243C2
:1007D000206572726F7200D4E0E9EB20EFEEE2F078
:1007E000E5E6E4E5ED210046696C652062726F6B19
:1007F000656E2100C1EBEEEA00426C6F636B00CDC9
:10080000E0E7E0E4004261636B00CDE5F2004E6F8B
:1008100000C4E00059657300CEF2ECE5EDE0004362
:10082000616E63656C00CFF0EEE4EEEBE6E8F2FC9F
:1008300000526573756D6500CFE0F3E7E00050612D
:1008400075736500D1F2EEEF0053746F7000000015
:1008500000000000005F00000007000700147F1484
:100860007F14242A7F2A12231308646236495522F2
:10087000500005030000001C2241000041221C0022
:10088000082A1C2A0808083E080800503000000802
:1008900008080808006060000020100804023E51AB
:1008A00049453E00427F4000426151494621414551
:1008B0004B311814127F1027454545393C4A4949A8
:1008C0003001710905033649494936064949291E4F
:1008D000003636000000563600000008142241148D
:1008E000141414144122140800020151090632495B
:1008F00079413E7E1111117E7F494949363E414181
:1009000041227F4141221C7F494949417F09090118
:10091000013E414151327F0808087F00417F41007C
:100920002040413F017F081422417F404040407FEA
:100930000204027F7F0408107F3E4141413E7F094F
:100940000909063E4151215E7F0919294646494958
:10095000493101017F01013F4040403F1F204020BD
:100960001F7F2018207F6314081463030478040396
:10097000615149454300007F414102040810204174
:10098000417F000004020102044040404040000159
:1009900002040020545454787F4844443838444476
:1009A0004420384444487F3854545418087E090180
:1009B00002081454543C7F0804047800447D40002D
:1009C0002040443D00007F10284400417F40007CCF
:1009D000041804787C0804047838444444387C14AF
:1009E000141408081414187C7C080404084854548F
:1009F0005420043F4440203C4040207C1C204020A8
:100A00001C3C4030403C44281028440C5050503C82
:100A10004464544C44000836410000007F0000004C
:100A20004136080008082A1C08081C2A0808143641
:100A3000773614007F3E1C08081C3E7F0004060722
:100A4000060410307030103E41081414413E00007E
:100A50000010387C101F081C3E0808000000000031
:100A60000000000000000000000000000000000086
:100A70000000000000000000000000000000000076
:100A80000000000000000000000000000000000066
:100A90000000000000000000000000000000000056
:100AA0000000000000000000000000000000000046
:100AB0000000000000000000000000000000000036
:100AC0000000000000000000000000000000000026
:100AD0000000000000000000000000000000000016
:100AE0000000000000000000000000000000000006
:100AF00000000000000000000000000000000000F6
:100B000000000000000000000000000000000000E5
:100B100000000000000000000000000000000000D5
:100B200000000000000000000000000000000000C5
:100B300000000000000000000000000000000000B5
:100B400000000000000000000000000000000000A5
:100B50000000000000000000000000000000000095
:100B600000000000000000000000000000007E11F6
:100B700011117E7F494949337F494949367F010137
:100B80000103E0514F41FF7F4949494177087F0800
:100B90007741494949367F1008047F7C2112097C3E
:100BA0007F0814224120413F017F7F020C027F7F9A
:100BB0000808087F3E4141413E7F0101017F7F09D6
:100BC0000909063E4141412201017F0101472810E8
:100BD00008071C227F221C63140814637F404040D6
:100BE000FF070808087F7F407F407F7F407F40FFEE
:100BF000017F4848307F4830007F007F48483022DE
:100C00004149493E7F083E413E462919097F20540B
:100C10005454783C4A4A49317C545428007C04049A
:100C2000040CE0544C44FC38545454186C107C10A0
:100C30006C44445454287C2010087C7C4122117C54
:100C40007C1028440020443C047C7C0810087C7CF8
:100C50001010107C38444444387C0404047C7C1418
:100C6000141408384444442004047C04040C5050F8
:100C7000503C3048FC483044281028447C404040D8
:100C8000FC0C1010107C7C407C407C7C407C40FC48
:100C9000047C5050207C5050207C7C5050200028F8
:100CA000445454387C10384438085434147C11248B
:100CB0001FBECFEFD0E1DEBFCDBF11E0A0E0B1E0BD
:100CC000E2E0FEEB00E00BBF02C007900D92AE31F8
:100CD000B107D9F72EE0AEE1B1E001C01D92A53B0E
:100CE000B207E1F70E94131B0C94FF5E89C91F92A3
:100CF0000F920FB60F9211240BB60F928F939F9302
:100D0000EF93FF93E0917605F09177050995FF91B8
:100D1000EF919F918F910F900BBE0F900FBE0F9090
:100D20001F9018950E94BF520E94B9528F930E9443
:100D3000B952982F8F9108950E94BF520E94B952C4
:100D40008F930E94B9528F930E94B9528F930E9441
:100D5000B952982F8F917F916F9108959F930E9420
:100D600007538F910C9407539F938F93862F0E9464
:100D70000753872F0E9407538F910E9407538F912B
:100D80000C940753F8E0E4E59091560AE90FF11D41
:100D9000808193959093560A09F00895F6E0E8EE65
:100DA000F093550AE093540A0895FCE0E5EB909126
:100DB000560AE90FF11D808193959093560A09F028
:100DC0000895F7E0E0E0F093550AE093540A08959F
:100DD000F9E0E4E59091560AE90FF11D80819395C1
:100DE0009093560A09F008959091570A9E7F909328
:100DF000570AF7E0E8E3F093550AE093540A0895A0
:100E0000FDE0E5EB9091560AE90FF11D8081939585
:100E10009093560A09F008959091570A9D7F9093F8
:100E2000570AF7E0E8E1F093550AE093540A089571
:100E30008091570A80FF0CC0F6E0E2ECF093550A6F
:100E4000E093540A8091540891E09093560A0895D3
:100E50008091300581608093300580912E059091BE
:100E60002F05019690932F0580932E0580E8089515
:100E70008091570A81FF0CC0F6E0E5EDF093550A2A
:100E8000E093540A8091B50C91E09093560A08952E
:100E90008091300581608093300580912E0590917E
:100EA0002F05019690932F0580932E0580E80895D5
:100EB000F8E0E4E59091560AE90FF11D80839395DF
:100EC0009093560A09F00895F7E0EEE7F093B40C1A
:100ED000E093B30C0895FCE0E5EB9091560AE90F1E
:100EE000F11D808393959093560A09F00895F7E0D9
:100EF000E6E9F093B40CE093B30C0895F9E0E4E56F
:100F00009091560AE90FF11D808393959093560AAC
:100F100009F008959091570A91609093570AF7E06D
:100F2000EDECF093B40CE093B30C0895FDE0E5EB29
:100F30009091560AE90FF11D808393959093560A7C
:100F400009F008959091570A92609093570AF7E03C
:100F5000EEEAF093B40CE093B30C08959091570A25
:100F600090FF0FC0809130058260809330058091A2
:100F70002E0590912F05019690932F0580932E05B5
:100F80000895F7E0E8E5F093B40CE093B30C809398
:100F9000540891E09093560A08959091570A91FF52
:100FA0000FC08091300582608093300580912E05BE
:100FB00090912F05019690932F0580932E0508950B
:100FC000F7E0EBE6F093B40CE093B30C8093B50C30
:100FD00091E09093560A08951DBC1CBCE091540A00
:100FE000F091550A099587FF04C01B981092840060
:100FF00008951B9A809107018093840008951DBC79
:101000001CBC8091AD07811118C0E091540AF09189
:10101000550A0995811102C00C94F836982F9F77D4
:101020009093AD0787FF06C01B9A809107018093BC
:10103000840003C01B98109284008091AD078150FA
:101040008093AD07089526B537B51DBC1CBC2F3F56
:1010500041E0340708F0C2C036952795422F8091B1
:101060000401813001F120F0823009F456C0AAC099
:1010700081E08093040180913F058F5F80933F055D
:1010800080914005909141059093430580934205DE
:10109000109241051092400582E10E94075384E3BB
:1010A0000E9407538FC080914605811105C02739E2
:1010B00018F02093460586C080914605882309F4E0
:1010C00081C0809146058695481708F07BC0209323
:1010D0003C0510921F0110921E0182E080930401D2
:1010E0008091470590914805A0914905B0914A0526
:1010F00020914B0530914C05820F931FA11DB11D0E
:101100008093470590934805A0934905B0934A05FD
:1011100010924C0510924B0555C0809144058111E9
:101120001BC083ED820F8A36B8F42A3518F4209359
:10113000440504C0822F869580934405C901880F19
:10114000991F63E070E00E94755960933E05822FFD
:10115000880F820F8093450580913E05481790F1D6
:1011600080914505841770F18091440543E0849F88
:10117000C001112495958795821793072CF48091CF
:101180001F01816080931F0180911E018F5F8093FA
:101190001E01883090F080911F010E9407538091BA
:1011A0004B0590914C05019690934C0580934B050F
:1011B00010921F0110921E0105C080911F01880F1F
:1011C00080931F012CB53DB580913D0590E08217BD
:1011D000930720F48CB59DB580933D050895A4E058
:1011E000B0E0E5EFF8E00C94735A8091040181308F
:1011F00009F44AC0823009F04AC00E940D53CE0162
:1012000001960E9488538091470590914805A091CE
:101210004905B0914A0580914B0590914C0560912C
:101220004705709148058091490590914A050E94B3
:10123000965380914B0590914C050E9407538091E5
:101240004B0590914C05892F0E9407530E940D5326
:1012500069817A818B819C810E9496538091470598
:1012600090914805A0914905B0914A050296A11DAB
:10127000B11D8093470590934805A0934905B0930D
:101280004A051092040103C083E080930401249670
:10129000E2E00C948F5A80E791E00C942F5208956D
:1012A000EF92FF921F93CF93DF9300D0CDB7DEB7BD
:1012B00089839A83F0DF89819A810E94E154182FF3
:1012C000882309F46EC010923F05109241051092D8
:1012D000400510924305109242051FBC9EB59368CD
:1012E0009EBD0E948C139EB5813011F4906401C0A4
:1012F0009F7B9EBD80E286BF97B7946297BF109296
:101300003D05109204011092470510924805109275
:10131000490510924A0510924C0510924B05109207
:101320004605109244050E9464137C010E94041338
:10133000970102C0369527958A95E2F7C9019695DF
:101340008795969587954FEF480F6AE070E00E9469
:101350006159461B409346050E9482137C010E94FE
:101360000413F70102C0F695E7958A95E2F7CF01DD
:101370009695879596958795809344052091440589
:10138000822F90E0880F991F63E070E00E947559EA
:1013900060933E0580914405982F990F980F909384
:1013A0004505812F0F900F90DF91CF911F91FF90F6
:1013B000EF900895A4E0B0E0E0EEF9E00C94735AE9
:1013C00087B78B7D87BF84E0809304010E947353AD
:1013D00069837A838B839C830E94615320913D05AE
:1013E000209146052091460520913C0520913C0521
:1013F0002091440520914405209120013091210144
:1014000069817A818B819C812496E2E00C948F5AC9
:101410000E94615387B78B7D87BF84E0809304016E
:10142000089580910401823041F480914B059091A0
:101430004C0590934105809340050E942E1388230C
:1014400069F080910401843049F0849B05C080914B
:1014500007018093840008951092840008958FE31B
:1014600095E00895809104010895CF931DBC1CBCA4
:10147000849B02C0C0E801C0C0E080914D05C81344
:1014800013C08091AD078F5F8093AD078091AD074A
:101490008F37F8F08091AD0790914D05890F0E942C
:1014A00007531092AD0715C08091AD0790914D057F
:1014B000890F0E940753CC2329F080910701809364
:1014C000840002C010928400C0934D0581E0809397
:1014D000AD07CF910895A2E0B0E0E1E7FAE00C9407
:1014E000725A89839A83D7DE89819A810E94E15456
:1014F000182F882309F162E477E581E496E534DC6E
:1015000081E090E02BDC84E49CEA28DC1092AD07BB
:101510001FBC1DBC1CBC2AE431E03BBD2ABD25E339
:101520003AE03093770520937605849B02C080E8EB
:1015300001C080E080934D05812F2296E3E00C945A
:101540008E5A849B02C080E801C080E080934D05E4
:101550000E94251CFC0114821582168287B78061C7
:1015600087BF81E08EBD0895A4E1B0E0EAEBFAE028
:101570000C94635A0E940D530E94535768E070E028
:1015800080E090E00E949653811102C0F12CF1C0DE
:101590000E9496526D877E878F87988B0E94245772
:1015A000282E8F77082F10E020E030E009831A837F
:1015B0002B833C8399E0892E912CA12CB12C312CCA
:1015C000412C512C320128E030E040E050E02D83E6
:1015D0003E834F835887C12CD12C76012D853E85C3
:1015E0004F85588982169306A406B50608F0AFC049
:1015F0000E942457B501A401517066277727452B17
:10160000462B472B09F4A895482F4F7750E060E010
:1016100070E009811A812B813C81040F151F261F60
:10162000371F09831A832B833C83822587FD05C0DE
:10163000C40ED51EE61EF71E84C014E7C11612E2C2
:10164000D106E104F10408F479C0A701960156958A
:1016500047953795279529873A874B875C87298156
:101660003A814B815C8124193509460957098985DE
:101670009A85AB85BC85281B390B4A0B5B0BA8EE02
:10168000B3E00E94DB5924E43CEA40E050E00E94D1
:10169000885929013A01C701B6012EEF30E040E038
:1016A00050E00E94885975016401C21AD30AE40A05
:1016B000F50AA70196018D819E81AF81B885281B0F
:1016C000390B4A0B5B0B298B3A8B4B8B5C8B33941E
:1016D0000E94435760E070E0CB010E94C35388230F
:1016E00009F454CF6D817E818F8198853DDB6989B6
:1016F0007A898B899C8938DBC301B20135DB0E9472
:101700000D530E945357C501B4016F5F7F4F8F4F38
:101710009F4F0E949653882309F438CF49805A80FE
:101720006B807C8009851A852B853C85401A510A7F
:10173000620A730ACD82DE82EF82F886C12CD12C38
:1017400076011FEF811A910AA10AB10A47CF0E94C0
:10175000435760E070E0CB010E94C353F82E88230A
:1017600009F414CF832D0E9407530E940D530E9449
:1017700053578F2D6496E2E10C947F5ACF93C82F74
:1017800097B79F7E97BF9EB59E7F9EBD10928400A7
:1017900080E00E94075389E10E94BB1F0E94C61F80
:1017A000C11103C0E1DEC82F01C0C1E00E94735324
:1017B0000E9461538C2F8170CF91089581E0DECF1C
:1017C0000895849B03C020E830E002C020E030E0B0
:1017D00040914D0550E081E02417350709F480E081
:1017E0000895A0E1B0E0E7EFFBE00C94665A6C01CD
:1017F0005B013A014901502E009719F480E090E016
:1018000065C061157105D1F383E08017BCF307FF54
:1018100005C080912A018111F1CF1DC080E108022D
:10182000F0011124E254FE4F9F2F990F990B80E194
:10183000E82EF12C8E010F5F1F4F9F01492F592F6A
:10184000692F792F892FF60109958823B9F28D81A7
:101850008111DFCFD3CF41E150E060E070E082E260
:1018600091E00E94285BD0922301C0922201B092A5
:101870002501A09224017092270160922601909286
:1018800029018092280157FC1CC08D8180932A0178
:10189000CE0109960E94A45160932B0170932C01F4
:1018A00080932D0190932E01CE010D960E94A4519C
:1018B00060932F0170933001809331019093320136
:1018C00003C08FEF80932A0182E291E06096EFE0FF
:1018D0000C94825A009721F0FC01108681E0089553
:1018E00080E00895843528F5603318F5262F269575
:1018F00026952695E82FF0E0962F977034E5239FE4
:10190000E00DF11D1124E455FA4FA1E0B0E0092EDD
:1019100001C0AA0F0A94EAF7442319F090819A2B88
:1019200003C0A09590819A239083262F482F0C9472
:1019300049350895CF93DF93D82FC62F8435E0F42F
:101940006033D0F4262F482F0E944935EC2FE695BE
:10195000E695E69584E5E89FF0011124ED0FF11D71
:10196000E455FA4FC77081E090E001C0880FCA9536
:10197000EAF7908198279083DF91CF910895A3E0B3
:10198000B0E0E5ECFCE00C94645A182F562E442E7F
:10199000C82ED12C1B821A824601840E911CA62EC1
:1019A000B12C3501620E711CEA81FB81EC0DFD1D2D
:1019B000E815F905DCF4E12CF12C3A80310EF70141
:1019C000EA0DFB1DE615F7055CF4652D6E0D402F45
:1019D000832D298387DF8FEFE81AF80A2981EFCF5B
:1019E000EA81FB813196FB83EA83DECF2150250D0E
:1019F0004FEF440D410F652D812F0E9449352396ED
:101A0000E1E10C94805AA0E0B0E0E9E0FDE00C9444
:101A1000685A182FB62E842EA22EE82EF12CC0E084
:101A2000D0E06701C40ED11C99249A94920E960EB0
:101A3000FE01EE0DFF1DEC15FD0564F47C2E710E0C
:101A4000402F6B2D872D4EDF402F692D872D4ADFCC
:101A50002196EECFEB2CF12CC0E0D0E06701CA0C50
:101A6000D11C8A94782C710EFE01EE0DFF1DEC1531
:101A7000FD0564F49C2E9B0C402F692D812F32DFD5
:101A8000402F692D872D2EDF2196EECF2FEF2A0DC7
:101A90002B0D482D410F6B2D812F0E944935CDB75D
:101AA000DEB7EDE00C94845AA0E0B0E0EAE5FDE09A
:101AB0000C946E5AD62EF82EC42FD0E0C80FD11D2C
:101AC000022F10E0060F111D2F2D30E02C173D07BF
:101AD0006CF4ED2C2E2D30E0201731072CF46E2DF8
:101AE0008F2D28DFE394F6CFF394EECFCDB7DEB79A
:101AF000E7E00C948A5A8FB9779BFECF77980895C8
:101B00008FEF8FB9779BFECF77988FB10895A4E0C0
:101B1000B0E0EDE8FDE00C94725A182F8FEF8FB90A
:101B2000779BFECF77988FB1812F80644C835B8346
:101B30006A837983E0DF7981872FDDDF6A81862FF1
:101B4000DADF5B81852FD7DF4C81842FD4DF11232F
:101B500021F0183039F487E801C085E9CCDF9AE03C
:101B60002FEF0AC08FEFFACF779BFECF77988FB118
:101B70008F3F21F4915011F02FB9F6CF2496E3E076
:101B80000C948E5AEF92FF920F931F938091350120
:101B900081111EC0209136013091370140913801EA
:101BA0005091390160913A0170913B01E12C82E042
:101BB000F82E0EE311E080913C0190913D0180D21E
:101BC000882321F081E08093350103C080E001C0CB
:101BD00081E01F910F91FF90EF900895A8E1B0E090
:101BE000E4EFFDE00C94635A29833A834B835C83D2
:101BF0006D837E838F8398874801FA8AE98A55240A
:101C00005A9469897A89672B09F41FC169807A809F
:101C100021E07222930140E050E060E070E0CB01EF
:101C200069863A874B875C876D877E878F87988B1D
:101C300029813A814B815C816D817E818F8198857C
:101C4000A984BA84C12CD12CE12CF12C00E010E045
:101C50000E94E65A288F3F8B4987452E6B8B7C8BE1
:101C60008D8B9E8B212C92E0392E261837084989BE
:101C70005A894215530508F41A01A0903601B09014
:101C80003701C0903801D0903901E0903A01F090CE
:101C90003B0100913C0110913D01288D3F89498510
:101CA000542D6B897C898D899E890E94EF5A29F475
:101CB00080913301882309F49FC064DF882309F4ED
:101CC000C6C0A8988091340182FF0FC0288D3F893B
:101CD0004985542D6B897C898D899E8909E00E94F4
:101CE000B55ABA01422F532F04C0488D5F896985C8
:101CF000742D81E10CDF882341F0A89AA8C0779B5E
:101D0000FECF77988FB18E3F11F05FB8F8CF8091FA
:101D100033018823A1F161147104A9F4211452E064
:101D2000350689F4F40180E090E05FB8779BFECF40
:101D300077982FB121930196811562E09607A9F754
:101D40007EEF971A48C09101260D371D80E090E084
:101D50005FB8779BFECF77984FB18615970548F00F
:101D60008217930730F4F4014083A4014F5F5F4F63
:101D70004A010196811552E0950751F72CC0EEE318
:101D8000F1E05FB8779BFECF77988FB1819363E0E6
:101D9000EE33F607B1F7788D709336018F89809313
:101DA000370199859093380140923901EB89E0938E
:101DB0003A01FC89F0933B012D8920933C013E8937
:101DC00030933D01B301625C7E4FA101C4010E94CA
:101DD0001F5B820C931C5FB8779BFECF77988FB107
:101DE0005FB8779BFECF77988FB1A89A5FB8779B43
:101DF000FECF77988FB109C0B301625C7E4FA1011D
:101E0000C4010E941F5B820C931C49895A894219A4
:101E100053095A8B498B910140E050E060E070E03B
:101E200080E090E0A980BA80CB80DC80ED80FE80ED
:101E30000F8118850E94D15A29833A834B835C8392
:101E40006D837E838F839887DCCE81E001C080E044
:101E50006896E2E10C947F5AA0E0B0E0E2E3FFE094
:101E60000C946D5ABA9AB99AA09ABB98A89A83E52D
:101E70008DB9709810923401CAE042DEC150E9F782
:101E8000A898C0E0D2E040E050E0BA0180E03FDE38
:101E9000813021F021972097B1F751C04AEA51E0F3
:101EA00060E070E088E033DE182F147082FD11C00E
:101EB00027DE26DE25DE80FF8DC022DE8A3A09F08D
:101EC00089C080913401826080933401C0E0D0E801
:101ED00025C040E050E0BA0187E319DE40E050E061
:101EE000BA0189E214DE82FDF1CF80913401816074
:101EF000EBCF81FD19C0C12CD12C760140E050E020
:101F0000BA0187E304DEB701A60189E200DE182FDB
:101F1000117080FF16C02197209789F080913401BD
:101F2000982F937031F706C0C12CD12CE12C30E4EE
:101F3000F32EE4CF40E050E0BA0181E0E7CFA89A69
:101F400048C0C0913401C1FF12C040E050E0BA0166
:101F50008AE3DDDD882311F0A89A3CC0D1DD86FF3D
:101F600003C0C460C0933401CBDDCADDC9DD40E0ED
:101F700052E060E070E080E1CADDA89A81112AC0D9
:101F80008DB18C7F8DB9709A8FEF809336018093DD
:101F90003701809338018093390180933A0180930F
:101FA0003B0180933C0180933D0181E080933501AA
:101FB000E12C22E0F22E0EE311E020E030E040E0E0
:101FC00050E060E070E080E090E008DE11E0811118
:101FD00001C010E0812FCDB7DEB7E8E00C94895A3C
:101FE000A2E1B0E0E6EFFFE00C94635A19012A0188
:101FF0006B837C838D839E8318870F833701DA82FE
:10200000C982BA86A9860115110511F480E054C071
:10201000E114F104D9F329813A812E153F05B0F37B
:1020200049855A85452B91F3970140E050E060E0E7
:1020300070E0CB01EB863C874D875E876F87788B9E
:10204000898B9A8B73010F8118859101A2016B8195
:102050007C818D819E81C2DD8823C1F27401810162
:1020600092014B815C816D817E818F819885E985AC
:10207000FA8509958823F9F09101A2016B817C8191
:102080008D819E81AB84BC84C12CD12CE12CF12CA0
:1020900000E010E00E94D15A19012A016B837C8371
:1020A0008D839E8329813A81261937093A832983B2
:1020B0002615370538F681E06296E2E10C947F5AE6
:1020C000A0E1B0E0E6E6F0E10C94635A29833A839C
:1020D0004B835C836D837E838F8398871E870D87F8
:1020E000FA86E98689859A85892B09F494C08981C5
:1020F0009A8191709C878B871C0129813A814B8141
:102100005C816D817E818F8198855101C12CD12C9C
:10211000E12CF12C00E010E00E94E65A288B3F876A
:102120003A011B012C01812C52E0952EEB85FC8598
:102130008E1A9F0A89859A858815990508F44C019D
:10214000A0903601B0903701C0903801D09039018D
:10215000E0903A01F0903B0100913C0110913D016B
:1021600028893F85A301B101C2010E94EF5A69F19C
:1021700009DD882309F459C0EB85FC85EF2BB9F400
:102180008114F2E09F0699F42889209336018F8507
:1021900080933701609238017092390120923A01A0
:1021A00030923B0140923C0150923D010EC0E12C27
:1021B00042E0F42E0EE311E028893F85A301B1012E
:1021C000C2010CDD8111E0CF30C0ED85FE85EE53FC
:1021D000F14089F4A8988091340182FF1EC02889BB
:1021E0003F85A301B101C20109E00E94B55ABA01BD
:1021F000422F532F15C0A4016D857E858B859C854C
:10220000825C9E4F0E941F5B1092350189859A85E2
:1022100088159905F9F681E051C048895F85B301B9
:1022200088E175DC882319F0A89A80E047C08EEF1A
:1022300062DC0EE311E0F80181918F015CDCF3E0D8
:102240000E331F07C1F78FEF56DC8FEF54DC2FEFF3
:102250002FB9779BFECF77988FB18F3FC1F78FB99A
:10226000779BFECF77988FB1A89A8D859E85880D34
:10227000991D9E878D87940140E050E060E070E0FA
:1022800080E090E0A980BA80CB80DC80ED80FE8089
:102290000F8118850E94D15A29833A834B835C832E
:1022A0006D837E838F839887E985FA85E819F9091C
:1022B000FA87E987F1E0F093350114CF6096E2E107
:1022C0000C947F5AABE0B0E0E8E6F1E10C94635A7D
:1022D00029833A83742E652E562E472E382E292EAA
:1022E0001D830C834701DF82CE82B986A886011543
:1022F000110511F480E061C02E813F81232BD1F3C1
:1023000031E03B83E114F10409F44AC01B8248C068
:102310008114910409F449C0E884F98409811A817F
:10232000272D362D452D542D632D722D8C819D81A9
:10233000EE81FF8109959B878A87892BB1F1FB810B
:10234000FF23A9F1EA84FB840C811D8129813A8154
:10235000472D562D652D742D832D922DB1DE8823AA
:1023600049F2EA84FB84970140E050E060E070E0CD
:1023700080E090E0A980BA80C72CD62CE52CF42C04
:10238000032D122D0E94D15A29833A83742E652E73
:10239000562E472E382E292E8A859B85881A990A13
:1023A0009B81992309F4B4CFB7CF81E006C02A8579
:1023B0003B858216930630F69DCF2B96E2E10C9476
:1023C0007F5AA0E0B0E0E7EEF1E10C946A5AEC012C
:1023D000009709F407C14DE150E060E070E00E9411
:1023E000285BA89840E050E0BA018AE090DB8111B8
:1023F00055C086DB8E3FE9F7DC2E0C2F1D2FB0E693
:10240000EB2EF12C7DDB402F4D1950E04F30510564
:1024100098F5FA01EA5BFF4F0C94C65988832CC0EB
:10242000F801808329C0F801818326C08A8724C0EF
:1024300090E0A0E0B0E00E2C04C0880F991FAA1F06
:10244000BB1F0A94D2F74B855C856D857E85482B32
:10245000592B6A2B7B2B4B875C876D877E870CC043
:102460008295807F8F8708C0282F22952F709F85A7
:10247000922B9F878F70888B0F5F1F4FF8E0EF1AAA
:10248000F10880EDE8168FEFF80609F0BBCF40E0C9
:1024900050E0BA0189E03BDB882311F0A89AA2C082
:1024A0002FDB8E3FE9F7D12CB12CE12CF12CC12C84
:1024B000912CAA24A39424DBD11007C0B82EB29487
:1024C000B694B694A3E0BA2286C09EE0D9120EC09C
:1024D00086FDA98E85FDAA8E84FDAB8E8C7090E062
:1024E00095958795959587958C8F75C0E1E0BE127F
:1024F00026C0F7E0DF1631F0DF1640F099E09D15B9
:1025000010F404C08F73FE2CEE24E82AE9E0DE12FA
:1025100062C0FFEFEF1AFF0A970140E050E060E071
:1025200070E080E090E003E10E949A5A298B3A8B98
:102530004B8B5C8B6D8B7E8B8F8B988F4CC0B110CF
:102540004AC097E0D916A9F19D1560F0E5E0DE16C6
:1025500069F1F6E0DF123FC08370E82EF12CFE2C0B
:10256000EE2439C099E0D91699F1D91640F1EAE084
:10257000DE1231C0881F8827881FC82A870120E003
:1025800030E0892D90E08C0D911D029604C0000F63
:10259000111F221F331F8A95D2F7098B1A8B2B8BA1
:1025A0003C8B1D8A1E8A1F8A188E15C08F70982E2C
:1025B00012C0E82AEE0CFF1CEE0CFF1C0CC082952A
:1025C000869586958370E82AFFEFEF1AFF0A03C00D
:1025D0008370C82ECC0CD39482E1D8126CCFA89A09
:1025E00081E001C080E0CDB7DEB7EBE00C94865A05
:1025F0008091510583700895E1E5F5E08370908145
:102600009C7F982B9083089580915105869586959F
:1026100083700895E1E5F5E08370880F880F90815D
:10262000937F982B908308958091510586FB88278E
:1026300080F90895E1E5F5E0908180FB96F99083BB
:1026400008958091510587FB882780F90895E1E579
:10265000F5E0908180FB97F9908308958091520571
:1026600081700895E2E5F5E0908180FB90F9908318
:102670000895809151058295837008958370282F65
:102680002295207F909151059F7C922B909351052C
:10269000813011F4D8980895811101C0D89A089515
:1026A00080916105909162050895909362058093F1
:1026B0006105089580915E0590915F05089590935E
:1026C0005F0580935E0508958091580590915905A6
:1026D00008959093590580935805089580915A055F
:1026E00090915B05089590935B0580935A0508953A
:1026F00080914E0590914F05089590934F058093DA
:102700004E05089580915605909157050895909330
:1027100057058093560508958091520586958170DE
:102720000895E2E5F5E0908180FB91F990830895AA
:10273000809153059091540508959093540580938A
:1027400053050895809350050C948F360895809119
:10275000500508958CEA9DE090935F0580935E0597
:1027600084EA96E090936205809361058BE692E09F
:1027700090935905809358058EEB90E090935B05FC
:1027800080935A0589EC90E090934F0580934E0515
:1027900084EF90E09093570580935605E2E5F5E0CD
:1027A00080818D7F80838FED97E090935405809397
:1027B000530510925D0510925C0580E580935005ED
:1027C000089542E050E060E070E081E595E00E940D
:1027D000085E90915105892F837092959370933084
:1027E00019F090E002976CF0B5DF80915105837F7E
:1027F0008093510582E042DF809151058C7F809368
:102800005105809151058295837038DF84E090E016
:102810000E94205E9C01245F31402D31354218F426
:10282000282F892F02C02CEA8DE020935E0580932B
:102830005F0586E090E00E94205E9C01245F3140AD
:102840002539314118F4282F892F02C024EA86E067
:10285000209361058093620588E090E00E94205EED
:102860009C01225331092F39374018F4282F892F22
:1028700002C02BE682E020935805809359058AE038
:1028800090E00E94205E9C0122533109273B334097
:1028900018F4282F892F02C02EEB80E020935A05D0
:1028A00080935B058CE090E00E94205E9C012253A7
:1028B0003109273B334018F4282F892F02C029EC17
:1028C00080E020934E0580934F058EE090E00E94BB
:1028D000205E9C0122533109273B334018F4282FF6
:1028E000892F02C024EF80E020935605809357057E
:1028F00080E190E00E94205E9C01205D37402536FB
:10290000310518F4282F892F02C02FED87E020937E
:1029100053058093540582E190E00E94205E803D43
:102920002AE8920724F0813345E794071CF020E061
:1029300080E002C0282F892F20935C0580935D05DD
:1029400083E190E00E94185E813808F080E5809372
:102950005005089542E050E060E070E081E595E0C8
:102960000E94255E60915E0570915F0584E090E0B5
:102970000E94455E609161057091620586E090E07D
:102980000E94455E609158057091590588E090E07D
:102990000E94455E60915A0570915B058AE090E067
:1029A0000E94455E60914E0570914F058CE090E06D
:1029B0000E94455E60915605709157058EE090E04B
:1029C0000E94455E60915C0570915D0582E190E03A
:1029D0000E94455E6091500583E190E00C94345E66
:1029E000089580E090E02091740027FD03C00197D6
:1029F0000097C9F708951092710088E480937000E1
:102A0000089584EA80937400ECDF90917100987FC0
:102A100081E0983009F080E00895CF9380FD02C0F6
:102A2000C8E101C0C0E48093730084E8809374001F
:102A3000D8DF40917100487F50E02C2F30E081E0DA
:102A40004217530709F080E0CF91089580937300F7
:102A500084E880937400C5DF90917100987F81E0D5
:102A6000983209F080E00895CF93DF93EC0184EC75
:102A700080937400B6DF9091710080917300888319
:102A8000987F81E0903509F080E0DF91CF91089543
:102A9000CF93DF93EC0184E880937400A2DF9091E0
:102AA0007100809173008883987F81E0983509F0E8
:102AB00080E0DF91CF91089584E98093740080E0F5
:102AC00090E02091740024FF05C001970097C9F79A
:102AD00080E0089581E008956AE070E088EE93E078
:102AE0000C946F500895CF939A9908C08091650512
:102AF0008F3F31F08F5F8093650502C010926505AE
:102B00009E9908C0809166058F3F31F08F5F80935A
:102B1000660502C0109266059B9908C08091630506
:102B20008F3F31F08F5F8093630502C01092630581
:102B30009D9908C0809164058F3F31F08F5F80932D
:102B4000640502C0109264059C9908C080916705D5
:102B50008F3F31F08F5F8093670502C01092670549
:102B600063DDC82F80916505853039F482E00E94CD
:102B7000372CCC2311F0B0DFC0E0809166058530A2
:102B800039F483E00E94372CCC2311F0A5DFC0E09C
:102B900080916305853039F480E00E94372CCC2386
:102BA00011F09ADFC0E080916405853039F481E04E
:102BB0000E94372CCC2311F08FDFC0E08091670595
:102BC000853029F484E00E94372CC11185DFCF9134
:102BD000089584B38C6784BB85B38C6785BB1092E2
:102BE00065051092660510926305109264051092B7
:102BF00067050895E82FF0E0ED59FA4F81E09081E4
:102C0000933308F480E00895A0E1B0E0EAE0F6E153
:102C10000C94635A782E698380916C05481720F0D4
:102C200090916D05941708F44EE290916E05911104
:102C30004EC0672CE42EF12CC72CD12C2981A22E5A
:102C4000B12C962D971980916A05981708F07FC1CD
:102C500020916C05B701621B7109869FA001879FB7
:102C6000500D1124490F511DE0916805F09169053F
:102C7000E40FF51F0491812C912C2601490E511C63
:102C800010E034E5431651040CF05EC194012A0DA6
:102C90003B1D203331050CF057C16981680D980147
:102CA000082C02C0359527950A94E2F720FF02C050
:102CB00041E001C040E0862D0E94720C8FEF881A1F
:102CC000980A98E089169104E1F66394BACF91309E
:102CD00009F092C040906B05469446944694439404
:102CE000E42EF12CE81AF10820916A05429E202D6D
:102CF00011242F5F2E9DC0012F9D900D1124E09176
:102D00006805F0916905E80FF91F24912A83242DA5
:102D100030E03D832C834F01E12CF12C272D30E056
:102D20003B872A873981232F30E03D872C876E2C03
:102D30003A81E31608F00AC100E010E0C12CD12C62
:102D400094012F5F3F4F3F832E832A853B852E0DB5
:102D50003F1D39872887670CEE81FF81EC0DFD1D33
:102D6000A4905980500E188A1F862C843D84200E12
:102D7000311EB12C28853985243531050CF0E4C08D
:102D80008F852F853889220D331D203331050CF0B6
:102D9000DBC020916B0530E04F855889400F511FF3
:102DA0004217530784F4D50102C0B595A7958A95BB
:102DB000E2F76F85650DA0FF02C041E001C040E071
:102DC000862D0E94720C2F8538892F5F3F4F388BDC
:102DD0002F872830310571F63FEFC31AD30A085FF9
:102DE0001F4FC41408F4B8CF8FEFE81AF80A2C81EB
:102DF0003D81820E931E9BCF923009F0A5C0909129
:102E00006B059695969596959F5F60916A05E42E61
:102E1000F12CE81AF108969F802D11248E9D9001C7
:102E20008F9D300D1124E0906805F0906905E20E49
:102E3000F31EAFEFA60F80E0462F50E0415051093E
:102E4000262E281AB42FB81B70E030E0F701E70FE8
:102E5000F11DE0813F5F7B0F3917C0F3E11105C021
:102E60008A1711F08F5FECCF212C00E010E0C12C0D
:102E7000D12C272D30E03D832C833981232F30E066
:102E80003F832E836980600E412C512C2E813F811F
:102E9000200F311F3B832A83342C421408F04AC090
:102EA00080916A058C9DF0018D9DF00D1124E40D3B
:102EB000F51DEE0DFF1D849019861886AC80BD802F
:102EC000A40CB51C912C370C84E5A816B104E4F5CC
:102ED00048856A817B8128853985620F731F60333D
:102EE000710594F560916B0570E0F901E00FF11F39
:102EF000E617F70794F4D40102C0B595A7954A9553
:102F0000E2F7622F660DA0FF02C041E001C040E081
:102F1000832D9E870E94720C9E85288539852F5FA0
:102F20003F4F398728872830310571F63FEF431A24
:102F3000530AB2CF8FEFC81AD80A085F1F4FC916BD
:102F400008F4A0CF822D03C080E001C08A81609682
:102F5000E2E10C947F5A0F931F93CF93DF93182FC6
:102F6000062FE62FF0E080916B052FE230E0281B62
:102F700031092E173F0754F0EA014991442331F0FB
:102F8000602F812F41DE8F5F180FF7CF812FDF91E8
:102F9000CF911F910F9108950F931F93CF93DF93BC
:102FA000182F062FE62FF0E080916B052FE230E01E
:102FB000281B31092E173F076CF0FA014491EF01ED
:102FC0002196442339F0602F812F1EDE8F5F180F6A
:102FD000FE01F4CF812FDF91CF911F910F910895C2
:102FE00087B78F7E87BF0E9491510E9461531092D4
:102FF00084001B9880913005882321F061E083E0F4
:10300000BDD703C081E080934003C0C70895CF922D
:10301000DF92EF92FF92CF93DF9300D000D0CDB735
:10302000DEB70E94AB54882309F488C00E9436574B
:103030000E949C06623579448644964409F07BC020
:103040000E949C060E949C06673571448645954403
:1030500009F071C00E949C0666367D468447904206
:1030600009F069C00E949C066031710581059105D7
:1030700009F061C00E949206019709F05CC00E94AD
:103080009206019709F057C00E949C069B01AC0173
:1030900069833A834B835C830E949C0629813A8131
:1030A0004B815C81261737074807590709F043C051
:1030B0000E9492060E9492060897E9F50E949C06DB
:1030C0006436714684479146B1F50E949C066B01B7
:1030D0007C011FBC60E074E284EF90E029813A81BA
:1030E0004B815C810E94885930937405209373054D
:1030F000C0926F05D0927005E0927105F092720552
:103100001DBC1CBC80917305909174059BBD8ABD4C
:103110008CEE97E0909377058093760580EF97E1AA
:103120009093C9078093C80787B7806187BF81E004
:103130008EBD80E004C054DF82E001C081E00F90CA
:103140000F900F900F90DF91CF91FF90EF90DF9055
:10315000CF900895A3E0B0E0E0EBF8E10C94735A4F
:103160004ADC4FDC8823F9F082EA57DC8823D9F067
:1031700080E06CDC8823B9F09FDC8823A1F041DC7F
:10318000882389F083EA49DC882369F0CE0103961D
:103190006BDC882341F0CE01029666DC882319F0AF
:1031A000CE01019675DC88DC8B81811106C08A8195
:1031B000811103C0898187FF1DC023DC811102C0FA
:1031C0007BDC18C082EA29DC8823D1F380E03EDC76
:1031D0008823B1F380E03ADC882391F380E036DC89
:1031E000882371F389818F7731DC882349F364DC8C
:1031F000882331F32396E2E00C948F5ACF93DF9328
:10320000EC01A8DFFEDB811103C056DC80E04BC07F
:1032100082EA03DC8823C9F382E018DC8823A9F35F
:103220004BDC882391F3EDDB882379F383EAF5DB2C
:10323000882359F3CE01059617DC882331F3CE019C
:10324000049612DC882309F3CE01039621DC88233F
:10325000E1F232DC8823C9F23D81232F26952695A1
:1032600026952E70922F990F990F920F3F70930F02
:103270009D833C81232F2695269526952E70922F8F
:10328000990F990F920F3F70930F9C833B81232FCF
:103290002695269526952670922F990F990F920FB5
:1032A0003F70930F9B83DF91CF9108951F93CF932E
:1032B000DF93EC014FDFA5DB811103C0FDDB80E074
:1032C00030C082EAAADB8823C9F382E0BFDB88230F
:1032D000A9F38D811AE0612F0E94555920E1829F48
:1032E000900D1124892FB2DB882341F38C81612F4B
:1032F0000E94555920E1829F900D1124892FA6DB51
:103300008823E1F28B81612F0E94555920E1829F31
:10331000900D1124892F9ADB882381F2CDDB88233D
:1033200069F2DF91CF911F910895CF93DF93EC0164
:1033300011DF67DB811103C0BFDB80E04BC082EA95
:103340006CDB8823C9F385E081DB8823A9F3B4DB38
:10335000882391F356DB882379F383EA5EDB8823A5
:1033600059F3CE01029680DB882331F3CE01079614
:103370007BDB882309F3CE01019676DB8823E1F21B
:10338000CE0186DB8823C1F297DB8823A9F23A813C
:10339000232F2695269526952670922F990F990F03
:1033A000920F3F70930F9A83398134FB222720F9C3
:1033B000220F922F990F990F920F3F70930F9983BD
:1033C0009881292F22952F709F703AE0239F900DAE
:1033D00011249883DF91CF9108951F93CF93DF93AA
:1033E000EC01B8DE0EDB811103C066DB80E040C07B
:1033F00082EA13DB8823C9F385E028DB8823A9F35D
:103400008A811AE0612F0E94555920E1829F900D18
:103410001124892F1BDB882341F34EDB882329F3FA
:10342000F0DA882311F382EAF8DA8823F1F287E0F0
:103430000DDB8823D1F28981612F0E94555920E14B
:10344000829F900D1124892F01DB882371F28881DE
:10345000612F0E94555920E1829F900D1124892FE0
:10346000F5DA882309F4C1CF27DB882309F4BDCF1F
:10347000DF91CF911F910895CF93DF93EC0155DF3A
:10348000882319F0CE01BADE01C080E08170DF919F
:10349000CF910895CF93DF93EC019FDF882319F03C
:1034A000CE0104DF01C080E08170DF91CF910895EB
:1034B0001F920F920FB60F9211240BB60F922F93FB
:1034C0003F934F935F936F937F938F939F93AF93AC
:1034D000BF93EF93FF930E94433CFF91EF91BF9105
:1034E000AF919F918F917F916F915F914F913F919C
:1034F0002F910F900BBE0F900FBE0F901F9018953D
:103500001F920F920FB60F9211240BB60F922F93AA
:103510003F934F935F936F937F938F939F93AF935B
:10352000BF93EF93FF930E942308FF91EF91BF9108
:10353000AF919F918F917F916F915F914F913F914B
:103540002F910F900BBE0F900FBE0F901F901895EC
:103550001F920F920FB60F9211240BB60F922F935A
:103560003F934F935F936F937F938F939F93AF930B
:10357000BF93EF93FF930E94EF08FF91EF91BF91EC
:10358000AF919F918F917F916F915F914F913F91FB
:103590002F910F900BBE0F900FBE0F901F9018959C
:1035A0001F920F920FB60F9211240BB60F922F930A
:1035B0003F934F935F936F937F938F939F93AF93BB
:1035C000BF93EF93FF9383B5845683BD80917505B8
:1035D0008160809375054CD1FF91EF91BF91AF91C0
:1035E0009F918F917F916F915F914F913F912F911B
:1035F0000F900BBE0F900FBE0F901F9018951F924B
:103600000F920FB60F9211248F939F9384B195B1AF
:1036100090937905809378059F918F910F900FBEBD
:103620000F901F90189585B7837E85BFA09A8F98BD
:10363000139A149A119A8C98D09A949A979A87E42C
:1036400087B98EEC86B98FEF9FEF909379058093C1
:1036500078050E9491510E9427572FE088E190E061
:103660000FB6F894A89581BD0FBE21BD66E970E044
:1036700088EE93E00E946F50E4D0A895A2D8A89558
:10368000B8D086E40E948F3662D80E948F360E949E
:10369000753564E670E080ED97E00E946F50A89564
:1036A00085B5856085BD87B7806887BF85E191E076
:1036B0000E94295260E070E0CB010E941F55A8953E
:1036C000789487DA9C993EC09A993CC09E993AC0FA
:1036D00062E370E088EE93E00E946F506EE170E06C
:1036E0008CED95E00E946F5064E170E080ED97E012
:1036F0000E946F506EE170E08CED95E00E946F507B
:1037000062E370E088EE93E00E946F5062E370E045
:103710008CEB92E00E946F508FEF809375059C991F
:1037200009C0A89568EE73E088EE93E00E946F50A0
:10373000A895F5CF9A9BF5CF9E9BF3CF1092A70546
:1037400082E119D41092750521D4A8950E943913ED
:10375000813009F0D89AC8EED3E037E4F32E4EEC6E
:10376000E42E0FEF1FEF8091750580FF3BC0809125
:1037700075058E7F80937505A895B5D90E9439137C
:10378000823071F483B38C778C3721F0D898C4EFF2
:10379000D1E006C0209721F02197209709F4D89A0C
:1037A0008091780590917905019681F08091780556
:1037B00090917905969587959695879580930701C1
:1037C000F7B8E6B8109379050093780580913E0329
:1037D000863020F48F5F80933E0304C010923E0336
:1037E0000E94DE340E94F9530E94623A0E94110A3C
:1037F000BACFB89ABA9ABD9AB99ABD9ABC9ABE9AEB
:10380000C59A80E58DB91EB80E94EB3668EA75E06E
:103810008CEA95E00E9496350C9475350895C5980C
:103820008FB98FEF779902C08150E1F7C59A08955B
:10383000C598C69880EA9FE00197F1F7C69AC59AA5
:1038400008958AE795E018CE08958AE795E00895EF
:10385000DC011196EC911197E23019F48C91837090
:1038600029F0F0E0EA58FE4F849108958DE1089523
:10387000CF93809180058F5F809380058436C0F15F
:103880001092800580917F058F5F80937F058C3338
:1038900078F110927F0580917E058F5F80937E0581
:1038A0008C3330F110927E0580917D058F5F80937F
:1038B0007D058831E8F010927D05C0917C05CF5FD1
:1038C000C0937C058AE795E0C3DF8C1788F491E00C
:1038D00090937C0580917B058F5F80937B058D3075
:1038E00038F090937B0580917A058F5F80937A05FD
:1038F000CF910895A8E0B0E0E0E8FCE10C94675AAD
:103900006C014B015A013901CE010196B5DD0E94CF
:1039100098132981820F911DF601918380838A81FA
:10392000F40180838B81F50180838C81F301808396
:103930008D81F80180838E81F70180832896EEE0E7
:103940000C94835A1092800510927F0510927E0588
:1039500010927D050895AC0167E280E01DCB0895CB
:10396000A0E0B0E0E6EBFCE10C94695A982E862EBC
:103970007A0105E010E0B12C40E0C0E1D7E28AE036
:10398000C82ED12CC701BE010E946159A62E61111B
:1039900005C0411103C0C130D10549F440E34A0DCF
:1039A000682D8B2D890D30D9B394B80E41E0AC9EB3
:1039B0009001AD9E300D1124E21AF30ACE01B6013A
:1039C0000E946159EB010150110901151105D1F651
:1039D0008B2DCDB7DEB7ECE00C94855AA1E0B0E0BA
:1039E000E4EFFCE10C94705A082FF62E842F6AE065
:1039F0000E94555940E3480F6F2D802F998304D9B9
:103A000011E0180F998140E3490F6F2D812F800F2E
:103A1000FBD88F5F810F2196E5E00C948C5A4F9272
:103A20005F926F927F928F929F92AF92BF92EF922E
:103A30000F93CF93DF934B015C0129013A01D02F03
:103A400060EF70E080E090E0A50194010E94885949
:103A5000C22F233008F4C3E0A0E3B0E0A301920139
:103A60000E94DB59A50194010E948859622FEC2F16
:103A7000F0E0E20FF11DF19714F060E36C1B01E040
:103A80002C2F4E2D8D2F0E94BF0CDF91CF910F91C7
:103A9000EF90BF90AF909F908F907F906F905F90CE
:103AA0004F9008958091A705833091F038F48823D2
:103AB00061F0813099F4C9DE01960895843059F09F
:103AC000853061F4C2DE05960895BFDE0296089542
:103AD000BCDE03960895B9DE0496089580E090E078
:103AE0000895CF93DF93EC010E94165B982F990FF6
:103AF000980F990FAE0167E284E5891B4DDADF91DB
:103B0000CF9108951F93CF93DF93EA01E82FF0E060
:103B10002091830530918405E217F307E0F0C90195
:103B20000596E817F907B8F4E21BF30B19E0E19FDB
:103B3000102D11241F5FAB01612F83E02DDACE0120
:103B40000E94165B982F990F980F990FAE01612F65
:103B500084E5891B21DADF91CF911F910895FF92AF
:103B60000F931F93CF93DF93D82FC92FF62E042FD7
:103B70000E94165B482F5BEF5403900111242C5ACE
:103B80003F4FE1E0F0E0E81BF1090E9FD0010F9FED
:103B9000B00D11242A0F3B1F37FF02C02F5F3F4F8C
:103BA00035952795122FED2FFC2F4491EF0121968B
:103BB000442339F06F2D812F27D8800F180FFE0175
:103BC000F4CFCDB7DEB7E5E00C948C5A0F931F937A
:103BD000CF93DF932091A705809183059091840571
:103BE000820F911D892B19F40E94235225C0C0E039
:103BF000D0E000E010E00E9423528C0F9D1FFC01DA
:103C000080812196811112C00F5F1F4F8091A705FF
:103C10002091830530918405280F311D0217130769
:103C200029F40E9423528C0F9D1F06C0C632F2E079
:103C3000DF0709F780E090E0DF91CF911F910F91AE
:103C4000089590918F05992391F0482F50E090911D
:103C5000A7052091830530918405290F311D421756
:103C6000530729F480919005909191050895823031
:103C700099F038F4882369F08130B9F40C9450132A
:103C80000895843079F058F0853079F40C948213DB
:103C900008950C945A1308950C94641308950C9489
:103CA0006E1308950C947813089580E090E00895C1
:103CB000A1E0B0E0EEE5FEE10C94655A182F7A0120
:103CC000482E512C209183053091840542165306CD
:103CD00008F472C0A9014B5F5F4F4416550608F007
:103CE0006BC0C201821B930B9C0189E0289F902C22
:103CF00011249394AB01692D83E04ED9812FA1DF6C
:103D0000482F892EC70149830E94165B6C014981A7
:103D1000E42FF82D05E010E0712C612C20E137E252
:103D20005AE0A52EB12CCF01B9010E946159611151
:103D300005C0611003C02130310519F47394662465
:103D40006394629FD001639FB00D1124EA1BFB0BAB
:103D5000C901B5010E9461599B010150110901156A
:103D6000110509F79601270D311D122F110F120FA2
:103D7000110F582D692D82E5811BF2DD8C5AA701A8
:103D8000692D811B09D980918F058823A9F0209185
:103D9000A7058091830590918405820F911D481697
:103DA000590651F469E0269F602D11246F5F4DE99B
:103DB00051E08CE4811BF0D82196E0E10C94815A0B
:103DC0000E9468520E94345460E070E0CB010E946F
:103DD0001F5510928405109283051092A70508952F
:103DE000CF92DF92EF92FF921F93CF93DF93CDB7E5
:103DF000DEB7A0970FB6F894DEBF0FBECDBF0E940E
:103E0000355230E040E051E0530FFC01E30FF11D6B
:103E100030813323C1F03F3229F4198220E0352F5D
:103E2000422FF1CF21E0240FE1E0F0E0EC0FFD1F85
:103E3000E40FF11D3083E1E0F0E0EC0FFD1FE20F35
:103E4000F11D1082ECCF0E945052182F882309F4E4
:103E50004BC00E9468520E943454CE0101960E94C9
:103E60003A566B017C0110928405109283051092E2
:103E7000A7058FEFC816D806E806F80671F10E946C
:103E80002652FC014281538164817581455051095C
:103E9000610971094C155D056E057F0508F50E94E5
:103EA0002652FC0182819381A481B5810697A105E8
:103EB000B10588F00E942652FC0142815381648141
:103EC00075814550510961097109C41AC092A7054D
:103ED0006A017B0105C0C092A705C12CD12C7601D7
:103EE000C701B6010E941F55812FA0960FB6F89406
:103EF000DEBF0FBECDBFDF91CF911F91FF90EF903E
:103F0000DF90CF900895FF920F931F93CF93DF938D
:103F1000EC01062F0E94695B8031A8F4482F5BEF0B
:103F20005403900111242C5A3F4F41E050E0481BAC
:103F30005109240F351F37FF02C02F5F3F4F3595C2
:103F40002795122F01C010E080E0FF24F394F80EB3
:103F5000FE01E80FF11D4081442341F0602F812FC5
:103F60000E9404168F5F180F8F2DEFCFCDB7DEB7ED
:103F7000E5E00C948C5A80934003089580938D055E
:103F80006093820583E1809340030895ACE1B0E043
:103F9000ECECFFE10C94635A80914003843129F4E6
:103FA00007B604FE02C00C94332C0FEF20E247E06A
:103FB00065E08EE498E00E9476360E948635809116
:103FC000400390E08A31910510F00C94312CFC01F3
:103FD000EB5AFF4F0C94C6590E94110A60E086E923
:103FE00095E091DF0E942F0AFC0100810E94F812E7
:103FF000811103C049EF57E002C044EF57E069E088
:1040000080E00E94CC17182F85E0810FBAE0EB2EDC
:10401000E10E013049F541E050E069E0A1DC1E2DE0
:10402000180F0E94320A813051F40E94F812811157
:1040300003C047E255E016C041E255E013C00E94BC
:104040002F0AFC014181528169E0812F89DC1E5FCA
:10405000180F0E94F812811103C04FE155E002C011
:104060004DE155E069E059C010E0A8014150510907
:1040700069E076DCE80E0E942F0AFC01438154813E
:1040800069E08E2D6DDCA2E0FA2EF80EFE0C0E9487
:10409000F812811103C04FE155E002C04DE155E037
:1040A00069E08F2D0E94CC170E94F812811103C085
:1040B00049EF57E002C044EF57E062E180E00E9420
:1040C000CC17F5E0FF2EF80EA80162E18F2D48DC39
:1040D00015E0180F1F0D0E94320A813051F40E9422
:1040E000F812811103C047E255E016C041E255E0E5
:1040F00013C00E942F0AFC014181528162E1812F8D
:104100002FDC1E5F180F0E94F812811103C04FE1CF
:1041100055E002C04DE155E062E1812F0E94CC17CD
:104120000E94F812811103C089E498E002C084E47F
:1041300098E011DC0E94110A0C94312C60E086E9B1
:1041400095E0E1DE01E027E044E56AE080E00E94DE
:10415000030D0E94333C9B01AC01A0E5B0E00E943E
:10416000DB592091890530918A0540918B0550914A
:104170008C050E948859422F23E06CE082E00E9467
:10418000BF0C8091BC07882309F444C00E94F81238
:10419000811103C049EF57E002C044EF57E063E1EB
:1041A00080E00E94CC17182F0E943C3C81110AC06D
:1041B0004091BC0750E063E185E0810FD1DB195FDE
:1041C000180F1CC042DBFC018681893138F09DEC60
:1041D000980F81E0983118F080E001C081E080FD07
:1041E000E7CF8091BC078A3010F4135F07C080913D
:1041F000BC07843610F41D5E01C0175E4FE263E118
:10420000812F0E940416810F4091BD0750E063E1A9
:104210008E5FA6DB0E943C3C882369F00E94F81266
:10422000811103C08EE398E002C088E398E041E08A
:104230006DE195DC31C00E94333C009189051091FD
:104240008A0520918B0530918C05601771078207D4
:10425000930768F4FADAFC011481F7DAFC010581AE
:10426000F4DAFC011083F1DAFC01018306C0EDDA17
:10427000FC011081EADAFC010181412F6DE18DE141
:10428000ADDB1DE1180F4AE36DE1812F0E9404169A
:10429000402F6DE1810FA2DB0E94333C0091890524
:1042A00010918A0520918B0530918C05601771075C
:1042B0008207930710F00C94E52B0E94F8128111ED
:1042C00003C089E498E002C084E498E044DB0E94E3
:1042D0003C3C0C94CD2B0E94F812811103C08AE85B
:1042E00097E002C080E897E041E061E038DC0E949E
:1042F000F812811103C08BE797E002C081E797E0D5
:1043000041E06AE02CDC0E94F812811103C088E6CB
:1043100097E002C08EE597E041E063E120DC0E9477
:10432000F812811103C086E597E002C08DE497E0A2
:1043300041E06CE114DC0E94F812811103C087E4B3
:1043400097E002C082E497E041E065E208DC0E9469
:10435000F8129091A70569E0969F602D112429E03D
:10436000811103C046E38FE002C040E48AE00E946E
:10437000540D0E942E57882311F40C94312C0E9466
:104380002E57482F50E060E080E0EADA0E94315773
:10439000AC016AE080E00BC141E060E080E695E0BE
:1043A000DEDB41E069E087E595E0D9DB40E062E1F2
:1043B00087E495E0D4DB41E06BE18DE395E0CFDB72
:1043C00040E064E28DE295E00C942F2C0E9426528E
:1043D000FC0182819381A481B581892B8A2B8B2B4F
:1043E00069F40E94F812811103C08AEB97E002C0C1
:1043F00082EB97E041E060E00C942F2CDD24D39415
:10440000CC24C394E12CF12C712C00E010E00E942C
:104410002352800F911FFC014081FBE0F71578F4D7
:104420000E942352800F911FFC018081882319F084
:104430000F5F1F4FF5CF01501109712C77C041114B
:1044400067C0FFEFEF1AFF0A0E942652A70160E043
:1044500070E0FC0182809380A480B58048155905E6
:104460006A057B0508F441C06091A70589E0689F53
:10447000602D112429E04DE480E00E94540D0E943B
:104480002652FC0182819381A481B5810697A10502
:10449000B10510F40C94312C00E020E343E060E01F
:1044A00081E50E94BF0C0E942652609183057091A5
:1044B0008405FC012681378140855185260F371FF1
:1044C000411D511D2C8F398F4A8F5B8F0E942652C0
:1044D000FC016281738184819581E2E0EE2E02E528
:1044E0002C8D398D4A8D5B8D57C22091830530917B
:1044F0008405C9010596E816F90608F0B5CF2E1512
:104500003F05A0F4F9E0CF0E712CDD24D3940EC04A
:104510008091830590918405E816F90638F06C2D9A
:104520008D2D0E940416D394D80E73940F5F1F4FE5
:10453000063222E0120708F46ACF96CF46E955E02A
:1045400060E080E00E94AB170E94F812811103C066
:1045500047EE57E002C047ED57E069E080E00E9477
:10456000CC1780919305833011F00C94312C0E946C
:10457000F812811103C049EF57E002C044EF57E041
:1045800064E180E00E94CC174091920550E064E124
:1045900083E2E6D915E2180F4FE264E1812F0E9411
:1045A00004164091BD0750E08E5F64E1810FD8D9B9
:1045B0000C94312C0E94F812811103C08AE895E016
:1045C00002C081E895E041E069E0C9DA0E94F81292
:1045D000811103C084E795E002C089E695E041E0DF
:1045E00062E1BDDA0E94F812811104C08FE198E007
:1045F0000C94142C88E198E00C94142C60E086E96B
:1046000095E081DC0E94F812811103C04AE055E078
:1046100002C043E055E069E080E00E94CC17182F0B
:104620000E942F0AFC01408150E069E085E0810F83
:1046300097D98090890590908A05A0908B05B090BD
:104640008C0508E010E0312C212C50E8C52E56E9ED
:10465000D52E58E9E52EF12C6AE0462E512C612C1E
:10466000712CC501B401A70196010E94885921113E
:1046700008C0211006C0F1E0CF16D104E104F10416
:1046800061F440E3420F62E1832D2C8F0E940416F7
:104690003394380E222423942C8DA22FB0E0A7014E
:1046A00096010E94DB59861A970AA80AB90AC7011F
:1046B000B601A30192010E94885969017A01015053
:1046C00011090115110569F615E0130D0E94F81284
:1046D000811103C047E155E002C042E155E062E1CB
:1046E000812F0E94CC1780919305823071F40E9433
:1046F000F812811103C047EE57E002C047ED57E0C2
:104700006BE180E00E94CC171BC08330C9F40E948B
:10471000F812811103C04DEC57E002C042EC57E0A3
:104720006BE180E00E94CC17182F4AE36BE10E94F6
:104730000416810F4091920550E06BE18B5F10D918
:104740000E94F812811104C085E098E00C94142CAA
:104750008FEF97E00C94142C0E94F812811107C07F
:104760000E94F81281110AC00DE616E00CC00E94EA
:10477000F812811106C005E616E005C009E616E04C
:1047800002C001E616E00E94F812811103C069E33D
:1047900077E002C064E377E0A80180E0B3D90E942B
:1047A0001413882339F00E94F81281110AC003E91A
:1047B00016E00CC00E94F812811106C00BE816E04A
:1047C00005C00FE816E002C007E816E00E94F812E4
:1047D000811103C06AE277E002C06FE177E0A801CF
:1047E00081E090D90E942113882339F00E94F812A9
:1047F00081110AC003E916E00CC00E94F812811171
:1048000006C00BE816E005C00FE816E002C007E896
:1048100016E00E94F812811103C064E177E002C043
:1048200069E077E0A80182E06DD90E942E13882309
:1048300039F00E94F81281110AC003E916E00CC099
:104840000E94F812811106C00BE816E005C00FE8BF
:1048500016E002C007E816E00E94F812811103C0BA
:104860006FEF76E002C065EF76E0A80183E04AD9F9
:104870000E943913882349F0813071F40E94F812A4
:10488000811111C003E916E016C00E94F8128111CF
:104890000DC00BE816E00FC00E94F812811109C08C
:1048A00002E816E008C00FE816E005C007E816E0C9
:1048B00002C00DE716E00E94F812811103C06BEEF2
:1048C00076E002C061EE76E0A80184E01BD90E9488
:1048D00004138150833048F4E82FF0E0EE0FFF1FFF
:1048E000E95EFE4F0081118102C00AE716E00E94D6
:1048F000F812811103C06BED76E002C062ED76E044
:10490000A80185E0FFD80E94F812811103C06AEC6B
:1049100076E002C061EC76E04BE951E086E0F2D847
:104920000E94F812811103C065EB76E002C068EACC
:1049300076E04BE951E087E0E5D80E94F81281115A
:1049400003C06FE976E002C066E976E04BE951E02A
:1049500088E0D8D86091A70589E0689F602D112470
:1049600029E042E582E00E94540D00E020E342E0AD
:1049700060E080E00E94BF0C8091A7052091830534
:1049800030918405280F311D40E050E0EE24E3947F
:104990006DE070E080E090E042D863C78091A705A9
:1049A000813009F4A1C038F0823009F4F6C08330B8
:1049B00009F463C107C20E94F812811103C08AEF93
:1049C00094E002C08DEE94E041E060E0C8D80E941F
:1049D000F812811103C08AEF94E002C08DEE94E0DA
:1049E0009F938F938E010F5F1F4F1F930F930E9412
:1049F000EC5B0E94FE562AE0A8010E94A45B6DE1D8
:104A000074E0C8010E94045B0E9411572AE0AE01C5
:104A10004F5E5F4F0E94A45BBE016F5E7F4FC80177
:104A20000E942F5B69E0C8016EDA0E94F8120F90B5
:104A30000F900F900F90811103C080EE94E002C0A0
:104A400082ED94E041E065E18AD80E94FB56BC010A
:104A50006F5F7F4FC8010E944E5B67E174E0C80141
:104A60000E94045B6BE174E0C8010E94045B0E9439
:104A7000FB56FC01808140E1BE016F5E7F4F90E0FC
:104A80000E949A5BBE016F5E7F4FC8010E942F5B40
:104A900069E174E0C8010E94045B6EE1C80133DA89
:104AA0000E94FB56FC0180894AE0B80190E00E9418
:104AB0009A5B6DE174E0C8010E94045B0E94FB56A2
:104AC000FC01878590E04AE0BE016F5E7F4F805316
:104AD000984F0E949A5BBE016F5E7F4FC8010E9493
:104AE0002F5B67E2C8016DC10E94F812811103C0FB
:104AF00084EC94E002C089EB94E041E060E02FD8C0
:104B00000E94FB56FC01638574858585968520E1AE
:104B1000AE014F5F5F4F0E94A45B69E0CE0101963A
:104B2000F2D90E94F812811103C084EB94E002C014
:104B30008EEA94E041E069E112D80E94FB56FC0144
:104B40002189328943895489658976898789908D3D
:104B500004E10E94B55AE22FA42FF52F2AE0AE01FE
:104B60004F5F5F4F6E2F732F8A2F9F2F0E94A45B82
:104B700067E174E0CE0101960E94045B0E94F81286
:104B8000811103C064E274E002C061E274E0CE010E
:104B900001960E94045B62E212C10E94F812811128
:104BA00003C080EA94E002C082E994E041E060E062
:104BB0000E94AF1D0E94FB5669E00496A4D90E9492
:104BC000F812811103C067E874E002C06DE774E079
:104BD000CE0101960E940F5B0E94FB56FC0182856C
:104BE00040E1BE016F5E7F4F90E00E949A5BBE0184
:104BF0006F5E7F4FCE0101960E942F5B62E1CE0176
:104C0000019681D90E94F812811103C085E794E0D2
:104C100002C08DE694E041E06BE10E94AF1D0E946E
:104C2000FB56FC01848D813059F028F0823069F008
:104C30008330A9F0C7C041E064E28EE594E01AC079
:104C400041E064E282E594E015C00E94F81281110F
:104C500003C088E494E00CC08AE394E009C00E9499
:104C6000F812811103C082E394E002C087E294E06D
:104C700041E064E20E94AF1DA5C00E94F8128111BC
:104C800003C08EEB93E002C087EB93E041E060E06D
:104C90000E94AF1D0E94855790E080319105E8F495
:104CA000FC01E159FF4F0C94C65982E194E021C008
:104CB0008FEF93E01EC086EF93E01BC080EF93E080
:104CC00018C08AEE93E015C080EE93E012C086ED26
:104CD00093E00FC089EC93E00CC00E94F8128111A0
:104CE00006C082E394E005C08CE094E002C087E255
:104CF00094E041E069E00E94AF1D0E94F81281112A
:104D000003C081EB93E002C089EA93E041E065E1F2
:104D10000E94AF1D0E94F812811103C06CE873E07D
:104D200002C063E873E0CE0101960E940F5B0E940F
:104D300074574AE0BE016F5E7F4F0E949A5BBE01CE
:104D40006F5E7F4FCE0101960E942F5B6EE1CE0118
:104D50000196D9D80E94F812811103C06FE973E05F
:104D600002C065E973E0CE0101960E940F5B0E94CC
:104D700063574AE0BE016F5E7F4F8130F0E29F07CC
:104D800050F40E949A5BBE016F5E7F4FCE01019688
:104D90000E942F5B13C0892F8695869590E00E9414
:104DA0009A5BBE016F5E7F4FCE0101960E942F5B22
:104DB0006FE174E0CE0101960E94045B67E2CE01D0
:104DC0000196A1D82091A70545E0249F90011124C8
:104DD000442737FD4095542FEE24E39403E564E126
:104DE00070E080E090E0D8CD0E94F812811103C0FD
:104DF00009E416E002C006E416E00E94F8128111F0
:104E000003C06EE378E002C068E378E0A80180E0C8
:104E10000E94581E0E94F812811103C009E416E096
:104E200002C006E416E00E94F812811103C069E294
:104E300076E002C063E276E0A80181E00E94581E9D
:104E40000E94F812811103C003E416E002C00FE3D0
:104E500016E00E94F812811103C067E376E002C0F9
:104E60006FE276E0A80182E00E94581E0E94F812CC
:104E7000811103C003E416E002C00FE316E00E94B4
:104E8000F812811103C06CE176E002C065E176E0C2
:104E9000A80183E00E94581E0E94F812811103C0ED
:104EA00003E416E002C00FE316E00E94F81281113D
:104EB00003C06EE076E002C067E076E0A80184E01F
:104EC0000E94581E0E94F812811103C003E416E0EC
:104ED00002C00FE316E00E94F812811103C062E0E5
:104EE00076E002C06BEF75E0A80185E00E94581ED5
:104EF0000E948C13813039F40E94F81281110AC08B
:104F000002E516E00CC00E94F812811106C00CE503
:104F100016E005C00CE416E002C007E516E00E94AA
:104F2000F812811103C063EF75E002C06CEE75E00A
:104F3000A80186E00E94821D0E94F812811103C020
:104F400065EE75E002C06AED75E04BE951E087E07F
:104F50000E94821D0E94F812811103C062ED75E06B
:104F600002C065EC75E04BE951E088E00E94821DCB
:104F700080918F0581110BC06091A70589E0689F22
:104F8000602D112429E042E582E00E94540D00E0EA
:104F900020E342E060E080E00E94BF0C80918F053A
:104FA00081115FC4E9CC0E94F812811103C086EB25
:104FB00095E002C08DEA95E041E069E00E94AF1DF6
:104FC0000E94F812811103C081EA95E002C086E9CF
:104FD00095E041E062E17EC102E010E040E3410F74
:104FE00061E0802F0E94041641E4410F6AE0802FA7
:104FF0000E9404164BE4410F63E1802F0E940416C7
:10500000163018F445E5410F0DC0163051F0173039
:1050100021F0183021F448E805C04FE503C047E807
:1050200001C04DE26CE1802F0E9404161F5F085FF3
:105030001A30A1F68091A705612F0E94555969E0A9
:10504000869F602D112429E049E0892F880F880F61
:10505000880F0E94540D41E867E280E00E94041628
:1050600046E955E067E28E5F0E94AB17182F0E9459
:10507000251CFC019681993120F09353983108F05A
:10508000F0C322E045E06DE2812F04C10E94251C9F
:105090008C018091A70581110AC043E861E08DE091
:1050A0000E94041644E86DE08DE00E940416F801A9
:1050B000428167E08AE00E94EE1C982F3BE0F32ECD
:1050C000F80E8091A705811109C02BE04EE065E044
:1050D0008DEF890F998F0E94540D998D4DE267E0F5
:1050E0008CE0890F0E9404168F0D23E0E22EE80E5B
:1050F0009091A705913069F496E0F92EF80E43E8F7
:1051000061E08F2D0E94041644E86DE08F2D0E940F
:105110000416F801418167E08E2D0E94EE1CE80E16
:10512000FF24F394FE0C8091A705813039F42BE025
:105130004EE065E083EF8E0D0E94540D4DE267E076
:1051400082E08E0D0E940416F80EB3E0DB2EDF0C19
:105150008091A705823069F443E861E0ACE0EA2E73
:10516000EF0C8E2D0E94041644E86DE08E2D0E94F7
:1051700004160E949813F8012081AC01420F511DC2
:1051800067E08D2D0E94B01C9091A705923041F4EC
:105190009AEE9F0D2BE04AE165E0890F0E94540DC5
:1051A0008091A705833051F443E868E182E10E94D1
:1051B000041644E864E282E10E940416F801438187
:1051C0006EE18FE00E94EE1CF0E1FF2EF80E909150
:1051D000A705933031F42BE04FE06CE18F5F0E9424
:1051E000540D4AE36EE18F2D0E9404168F0DFF24AB
:1051F000F394F80E9091A705943069F4E4E0EE2E54
:10520000E80E43E868E18E2D0E94041644E864E24B
:105210008E2D0E940416F80144816EE18F2D0E94AC
:10522000EE1C8F0DFF24F394F80E9091A705943097
:1052300031F42BE04FE06CE18E500E94540D4AE3B4
:105240006EE18F2D0E940416F80EDD24D394DF0C3E
:105250008091A705853069F443E868E174E0E72EA2
:10526000EF0C8E2D0E94041644E864E28E2D0E94FD
:105270000416F80145816EE18D2D0E94EE1C90917F
:10528000A705953009F0EDC293EF9F0D2BE04FE09D
:105290006CE1890F0E94540DE4C260E086E995E05C
:1052A0000E94831F0E94F812811103C084E793E0DB
:1052B00002C085E693E041E062E10E94AF1D0E94DA
:1052C000F812811103C089E593E002C08BE493E0FA
:1052D00041E06BE10E94AF1D0E94F812811103C0F2
:1052E0008EE098E002C08AE098E00E94AB1C0E9429
:1052F000F812811103C084E198E064C281E198E072
:1053000061C20E94F812811103C08BE997E019C0B5
:105310008FE897E016C00E94F812811103C082E85E
:1053200092E002C089E792E041E069E00E94AF1D8F
:105330000E94F812811103C081E792E002C084E666
:1053400092E041E062E18BC20E94F812811103C039
:1053500082E493E002C084E393E041E069E00E94CC
:10536000AF1D0E94A713482F50E067E185E20E941D
:10537000B01C01E028E040E460E28AE00E94BF0C3B
:1053800070C20E94F812811103C08EE293E002C045
:1053900087E293E041E062E00E94AF1D2BE044E52C
:1053A00060E080E00E94540D80918D05833009F407
:1053B00051C028F4813049F08230F1F0ADC0843022
:1053C00009F490C0853079F1A7C00E94F8128111CC
:1053D00003C08AE193E002C08AE093E041E060E12B
:1053E0000E94AF1D0E94F812811103C085E093E076
:1053F0008FC080E093E08CC00E94F812811103C03E
:1054000085EF92E002C083EE92E041E060E10E940D
:10541000AF1D0E94F812811103C08EED92E078C09A
:1054200089ED92E075C00E94F812811103C08DECE5
:1054300092E002C08BEB92E041E060E10E94AF1D80
:105440000E94F812811103C086EB92E061C081EBEB
:1054500092E05EC090913005892F827090FF16C057
:10546000882351F00E94F812811103C081E392E079
:1054700018C085E292E015C00E94F812811103C0A5
:1054800088E192E00EC089E092E00BC0882369F0C9
:105490000E94F812811103C08BEF91E002C08CEEE4
:1054A00091E041E060E10E94AF1D4AE0BE016F5F04
:1054B0007F4F80912E0590912F050E949A5B0E944C
:1054C000F812811103C064EE71E002C06CED71E06E
:1054D000CE0101960E94045B69E1CE0101960E9413
:1054E000831F1AC00E94F812811103C086EA92E05D
:1054F00002C086E992E041E060E10E94AF1D0E9497
:10550000F812811103C08FE892E002C089E892E0AE
:1055100041E069E10E94AF1D01E020E344E560E065
:1055200080E00E94030D9DC10E94F812811103C00A
:1055300086E492E002C08DE392E041E062E00E94E6
:10554000AF1D6BE032C00E94F812811103C08CE5E0
:1055500092E002C08EE492E041E062E00E94AF1D62
:105560002BE044E560E080E00E94540D01E020E380
:1055700044E560E080E00E94030D41E060E183EAE1
:1055800091E00E94AF1D41E069E18FE991E00E9446
:10559000AF1D6091A70589E0689F602D1124615FB0
:1055A00029E042E289E176CE60E086E995E00E945A
:1055B000831F57C160E086E995E00E94831F01E0E8
:1055C00027E044E56AE080E00E94030D0E9447372F
:1055D000882389F00E94251CFC01F4800E94251C70
:1055E000FC0105810E94251CFC01F0820E94251C03
:1055F000FC01018308C00E94251CFC01F0800E9470
:10560000251CFC01018110E0FCE3FF9E000D111D33
:1056100011240E94251C44E6409F9001419F300DBB
:105620001124FC018681A901480F511DCA010E9465
:10563000D63820E5209FC001219F900D1124609154
:105640009405709195050E946159462F01E023E071
:105650006CE082E00E94BF0C8091BC07882309F4B3
:1056600047C00E94F812811103C049EF57E002C001
:1056700044EF57E063E180E00E94CC17182F80913F
:10568000AC0781110BC04091BC0750E063E185E09D
:10569000810F0E94B01C195F180F1DC00E94251CAD
:1056A000FC018681893138F09DEC980F81E09831BA
:1056B00018F080E001C081E080FDE5CF8091BC075B
:1056C0008A3010F4135F07C08091BC07843610F451
:1056D0001D5E01C0175E4FE263E1812F0E94041638
:1056E000810F4091BD0750E063E18E5F0E94B01CC6
:1056F0008091AC07882371F00E94F812811103C0D9
:105700008EE398E002C088E398E041E06DE10E94FA
:10571000AF1D2EC00E944737882389F00E94251CA8
:10572000FC0114810E94251CFC0105810E94251C9E
:10573000FC0110830E94251CFC01018308C00E940B
:10574000251CFC0110810E94251CFC010181412FB8
:105750006DE18DE10E94EE1C1DE1180F4AE36DE141
:10576000812F0E940416402F6DE1810F0E94EE1CD4
:105770000E944737811104C08091AC07882329F12A
:105780000E94F812811103C089E498E002C084E409
:1057900098E00E94AB1C8091AC07882351F00E94D6
:1057A000F812811103C081E398E00CC086E298E012
:1057B00009C00E94F812811103C08EE398E002C074
:1057C00088E398E00E94711D4CC00E94F81281117C
:1057D00003C08DEA97E002C086EA97E041E067E205
:1057E0003EC060E086E995E00E94831F0E94251C70
:1057F000FC01058144816DE18DE10E94EE1C1DE1FB
:10580000180F4AE36DE1812F0E940416402F6DE1CD
:10581000810F0E94EE1C0E94F812811103C089E4DE
:1058200098E002C084E498E00E94AB1C1AC00E9479
:10583000F812811103C085ED91E002C08BEC91E07C
:1058400041E060E10E94AF1D0E94F812811103C087
:1058500083EC91E002C086EB91E041E069E10E94B7
:10586000AF1D0E949C366C96E2E10C947F5A8F9299
:105870009F92AF92BF92CF92DF92EF92FF92CF931F
:10588000DF93C82F4091400350E04931510508F0A3
:10589000F5C7FA01E158FF4F0C94C659823009F060
:1058A000EDC70E94DA096093890570938A05809399
:1058B0008B0590938C0562E975E086E995E00E947E
:1058C0000E3988E080934003D9C70E94333CC090D2
:1058D0008905D0908A05E0908B05F0908C056C15B9
:1058E0007D058E059F05B0F0C250C23008F0C6C7D6
:1058F00080913005882351F083E080938D0581E00D
:105900008093820583E180934003B8C781E0809350
:105910004003B4C7C13009F442C078F1C23019F075
:10592000C33009F1ABC70E94D93B609185057091E6
:10593000860580918705909188050E941F5580916A
:105940003005882341F083E080938D0581E08093CA
:10595000820583E101C081E0809340030E942652CA
:105960000E9426528BC70E943C3C811103C00E94BA
:10597000EE3B84C70E94F93B81C70E943C3C8823D0
:1059800009F47CC79091BC078091BD07981708F077
:1059900075C78091BC078F5F8093BC076FC70E945B
:1059A0003C3C882309F46AC78091BC07823008F424
:1059B00065C78091BC0781508093BC075FC7813069
:1059C00091F028F0C350C23008F058C717C080913A
:1059D000A705882321F081508093A7054FC784E055
:1059E0008093A7054BC78091A705843020F48F5F73
:1059F0008093A70543C71092A70540C78091A705CC
:105A000081110CC0879906C081E0809340030E94F9
:105A1000E01E34C781E18093400330C7813041F4F8
:105A20008799F8CF85E1809340031092A70526C798
:105A3000823051F484E080934003109284051092E8
:105A400083051092A7051AC7833099F480E18093EB
:105A500040030E94C61F879908C089E080934003D5
:105A60001092A7050E94975609C781E180934003D1
:105A700005C7843009F002C785E080934003FEC665
:105A800010924003FBC60E942652FC0142815381C2
:105A900064817581452B462B472B49F40E94F01EEB
:105AA0008111ECC6109240031092A705E7C6C11100
:105AB00065C08091A70581115DC08091830590919B
:105AC0008405009731F001979093840580938305B6
:105AD000D5C60E942652FC0186819781A085B1859A
:105AE000892B8A2B8B2B09F4C9C60E942652FC01F4
:105AF00080809180969487940E942652A12CB12C8C
:105B00002091830530918405FC0186819781A085D1
:105B1000B185820F931FA11DB11D88169906AA0693
:105B2000BB06A0F40E942652209183053091840583
:105B3000FC01C680D780E084F184C20ED31EE11C34
:105B4000F11CC818D908EA08FB0803C0C12CD12CE5
:105B500076010E942652FC018681978101978C195B
:105B60009D099093840580938305C701B6010E9427
:105B70001F5584C681508093A70580C6C13009F0A7
:105B8000A6C08091A705C0908305D0908405C80E5B
:105B9000D11CE12CF12C0E942652FC0182819381C0
:105BA000A481B5810197A109B109C816D906EA06F1
:105BB000FB0608F063C68091A705843020F48F5F50
:105BC0008093A7055BC6C0918305D09184050E9490
:105BD0002652FC01808191810597C817D90750F49E
:105BE000809183059091840501969093840580931C
:105BF000830544C60E942652FC01C680D780E084FB
:105C0000F1840E942652FC0180819181C80ED91E28
:105C1000E11CF11C0E942652FC0182819381A48127
:105C2000B5810197A109B1098C159D05AE05BF0588
:105C300008F424C60E942652FC018080918096942C
:105C400087940E942652A12CB12C2091830530917B
:105C50008405FC0186819781A085B185820F931F01
:105C6000A11DB11D88169906AA06BB06A0F40E94C4
:105C700026522091830530918405FC01C680D7808F
:105C8000E084F184C20ED31EE11CF11CC818D908AF
:105C9000EA08FB0803C0C12CD12C7601C091830512
:105CA000D09184050E9426529E012F5F3F4FFC0138
:105CB00086819781280F391F2C193D09309384055F
:105CC00020938305C701B6010E941F55D7C5C23076
:105CD00009F4E4CEC33009F04DC00E94E61DEC018A
:105CE00088818E3379F480E1809340030E94C61F3F
:105CF000CE0101960E9438520E94E01E81E08093FE
:105D00004003BCC50E9426520E942652CE010E942A
:105D1000695B843008F4B2C59E01280F311DF9017A
:105D2000349720812E3209F0A9C531963081306236
:105D3000319620812062319680818062343739F437
:105D4000213609F09BC5803709F098C5CAC5373799
:105D500039F4213609F092C5863709F08FC59BC505
:105D6000323609F08BC5213609F088C5873709F02E
:105D700085C5FDC5C43009F081C50E94E61D2EE031
:105D80002093400340E150E0BC0186E995E00E9489
:105D9000555B74C581E08093400370C5823009F083
:105DA0006DC580918E05813019F40E94080A04C0E7
:105DB000823011F40E94DE0B1092400381E0809348
:105DC000A7055CC581E08093A705809130058823F5
:105DD00049F083E080938D051092820583E18093E2
:105DE00040034CC51092400349C5813009F48EC070
:105DF00008F477C0823019F0833041F03FC58093BA
:105E0000A705109240030E94AA1438C52091A70547
:105E10008091830590918405820F911D89309105B1
:105E200008F02CC5FC01E856FF4F0C94C6590E949F
:105E3000F81291E0811190E0892F0E94FC121EC59A
:105E40000E94141391E089270E941A1317C50E941B
:105E5000211391E089270E94271310C50E942E1359
:105E600091E089270E94321309C50E9439138111DC
:105E700004C081E00E943E1301C50E9439138130A5
:105E800021F482E00E943E13F9C480E00E943E1398
:105E9000F5C40E940413833021F480E00E940A13A9
:105EA000EDC40E9404138F5F0E940A13E7C48AE0C6
:105EB0008093400310928F051092A70510928405DD
:105EC00010928305DBC48DE0809340030E94251C63
:105ED0000E943C1A1092A705D1C482E1809340032E
:105EE000CDC48091A705882321F081508093A70518
:105EF000C5C48091830590918405009709F4BEC4C0
:105F000001979093840580938305B8C48091A70579
:105F1000843020F48F5F8093A705B0C480918305FF
:105F2000909184058430910508F0A8C4019690935F
:105F3000840580938305A2C4813009F4ADC008F4C0
:105F400074C0823019F08330A1F098C480918F051D
:105F5000882319F010928F0591C482E090E090930D
:105F600084058093830584E08093A7058093400394
:105F700085C480918305909184054091A7059C017B
:105F8000240F311D2630310509F442C060F027305E
:105F9000310509F446C02830310509F06FC48BE0A3
:105FA000809340036BC490918F05242F280F992371
:105FB00021F18091900590919105223099F038F46B
:105FC000222369F02130B1F40E94551313C024300C
:105FD00079F058F0253071F40E9487130BC00E94AD
:105FE0005F1308C00E94691305C00E94731302C0AA
:105FF0000E947D1310928F0541C4822F0E94211EA2
:10600000909391058093900581E080938F0536C42D
:106010000E948C1391E0811190E0892F0E949113CE
:106020002DC487E08093400329C480918F0520917F
:10603000A7058823F1F08091900590919105019634
:106040009093910580939005E0918305F0918405EC
:10605000E20FF11DEE0FFF1FED57FE4F259134911A
:106060002817390708F00AC430939105209390054A
:1060700005C4222321F021502093A705FFC380915E
:10608000830590918405009709F4F8C301979093D4
:10609000840580938305F2C380918F052091A70525
:1060A0008823F1F08091900590919105019790934C
:1060B000910580939005E0918305F0918405E20FAE
:1060C000F11DEE0FFF1FE157FE4F2591349182170E
:1060D000930708F0D3C33093910520939005CEC366
:1060E000243020F42F5F2093A705C8C38091830537
:1060F000909184058430910508F0C0C30196909377
:10610000840580938305BAC3823061F48AE080936A
:10611000400384E090E0909384058093830580930E
:10612000A705ACC3833009F0A9C38AE0809340037C
:1061300084E090E090938405809383058093A70585
:106140000E94AA139BC3882319F0813051F012C01A
:106150008091A705882309F491C381508093A705F6
:106160008DC38091A705833008F088C38F5F80932B
:10617000A70584C383E08093A705109240037EC3E4
:10618000823059F028F48823D1F0813019F176C398
:10619000833061F0843051F171C38091A705882369
:1061A00009F46CC381508093A70568C38091A7054B
:1061B000873208F063C38F5F8093A7055FC3809128
:1061C000A7058A508093A705853608F457C3109217
:1061D000A70554C38091A705865F8093A7058832E1
:1061E00008F44CC387E28093A70548C386E995E08D
:1061F0000E94695B9C015091A705563249F488239F
:1062000009F43CC3F901FF27EB56FA4F108236C35D
:10621000573209F08FC0811106C081E08093A70535
:10622000109240032BC380918E05813019F461EBED
:1062300071E009C0833019F46CEA71E004C0823067
:1062400031F467EA71E086E995E00E94045B89E138
:10625000809340030E94C61F0E944B090E9468520F
:106260000E94345486E995E00E949F52882321F0D1
:106270008FE08093400302C3C0918E05C130E1F4EA
:1062800086E995E00E945009811112C086E995E0E7
:106290000E94695B99278E569A4FFC011082C09329
:1062A0008D058CE08093820583E180934003E6C2F4
:1062B00087E080934003E2C2C330E1F486E995E0D1
:1062C00063D4811113C086E995E00E94695B992728
:1062D0008E569A4FFC01108281E080938D058CE0F0
:1062E0008093820583E180934003C8C287E0809356
:1062F0004003C4C2C23009F0C1C286E995E00E94E1
:106300006B0A811113C086E995E00E94695B9927A9
:106310008E569A4FFC01108281E080938D058CE0AF
:106320008093820583E180934003A8C287E0809335
:106330004003A4C28C3008F0A1C23327EAE0852FC5
:106340006E2F0E945559492F852F0E945559813033
:1063500041F028F0823041F0833041F017C090E3E3
:1063600001C091E4940F15C09BE4FCCF463010F4BB
:1063700095E5F8CF463061F0473021F0483021F400
:1063800098E807C09FE505C097E803C090E001C00A
:106390009DE2F901EA56FA4F908311826FC2823072
:1063A00069F030F4882319F1813009F461C066C2C4
:1063B000833091F0843009F495C060C224E02093CA
:1063C000400383E090E090938405809383052093BD
:1063D000A7050E94AA1452C28091A705853020F417
:1063E0008F5F8093A7054AC21092A70547C280918C
:1063F000A705823001F50E949813EC010E94251C2C
:10640000FC018081C80FD11DC433F8E0DF0708F418
:1064100021960E949813C81BD90BC430D10530F0C7
:1064200024970E94981304960E949D130E94251C95
:10643000FC01C08318C0813029F030F0833051F066
:10644000CBE309C0CCE007C00E94251C0E94281C99
:10645000C82F01C0C7E10E94521DFC0180818C172A
:1064600010F48F5F80830E94251C0E944A1A06C286
:106470008091A705823009F50E949813EC010E94D3
:10648000251CFC018081C80FD11DC03EF7E0DF074D
:1064900008F021970E949813C817D90730F40E947A
:1064A000981304970E949D1324960E949813C81B6A
:1064B000D90B0E94251C2C2F0EC00E94521D30911A
:1064C000A705FC012081313019F0211103C005C05E
:1064D000223018F02150FC0120830E94251C0E94CC
:1064E0004A1ACCC10E94251CFC0185818F3168F0BD
:1064F0000E94251C2BE3FC0125830E94251C23E61A
:10650000FC0126830E94381C04C00E94251CFC014B
:1065100015820E94251C0E944A1AB0C1823009F0DF
:10652000ADC181E080934003A9C1823019F083306E
:1065300071F0A4C186E995E00E94695B99278E56A7
:106540009A4FFC0110828CE08093400397C1C09168
:106550008E05C130E1F486E995E00E945009882358
:1065600021F087E08093400389C186E995E00E948D
:10657000695B99278E569A4FFC011082C0938D0556
:106580008CE08093820583E18093400377C1C23021
:1065900009F074C186E995E00E946B0A882321F016
:1065A00087E0809340036AC186E995E00E94695BB9
:1065B00099278E569A4FFC01108281E080938D05B9
:1065C0008CE08093820583E18093400357C1109251
:1065D000400354C10E94A713C130F1F030F0C23023
:1065E00009F448C0C330E1F049C187FD0EC08F5F98
:1065F0000E94A2138091A705811140C166E970E055
:1066000088EE93E00E946F5039C16CED75E088EE22
:1066100093E00E946F5032C18823B9F38150E8CFD4
:106620000E94AA148091A705811124C062E370E042
:106630008CEB92E00E946F5062E370E088EE93E092
:106640000E946F506EE170E08CED95E00E946F50FB
:1066500064E170E080ED97E00E946F506EE170E0C1
:106660008CED95E00E946F5062E370E088EE93E05D
:106670000E946F508091A705811103C010924003C2
:10668000FDC084E080934003F9C080918D05833084
:1066900031F410922F0510922E0510923005809142
:1066A000820580934003EAC08130E1F090F08230AF
:1066B00001F1833009F0E2C08091A7058F5F8093DC
:1066C0008E051092A7058CE08093400310929605EA
:1066D000D5C08091A705882309F4D0C0815080934C
:1066E000A705CCC08091A7058111C8C0C093A7059C
:1066F000C5C01092400381E08093A705BFC08ED231
:1067000081E08093A70580913005882349F083E0DC
:1067100080938D051092820583E180934003AEC083
:1067200010924003ABC081E08093A70580E00E94F7
:10673000BE0B811109C085E080938D051092820502
:1067400083E1809340039AC080913005882349F00B
:1067500083E080938D051092820583E1809340034E
:106760008DC0109240038AC0813009F47AC008F4C9
:1067700068C0823019F0833001F180C088D3811164
:1067800037D360918505709186058091870590913A
:1067900088050E941F5580913005882351F083E0C1
:1067A00080938D0581E08093820583E1809340038F
:1067B00065C081E08093400361C00E943A57811117
:1067C00018C060918505709186058091870590912C
:1067D00088050E941F5580913005882339F0C093A9
:1067E0008D0581E08093820583E101C081E0809383
:1067F00040038091AC07811112C00E94251CEC015E
:106800000E94251CFC01848188830E94251CEC01C8
:106810000E94251CFC018581898347D42FC04FD459
:106820000E94251CEC010E94251CFC0180818C83A8
:106830000E94251CEC010E94251CFC0181818D8396
:106840001DC025D381111AC09091BC078091BD074E
:106850009817A0F48091BC078F5F8093BC073AD44F
:106860000DC015D381110AC08091BC07823030F071
:106870008091BC0781508093BC072CD40E94C61F16
:10688000DF91CF91FF90EF90DF90CF90BF90AF90CE
:106890009F908F90089584E18093400341E150E000
:1068A000BE0186E995E00E94555B0E94C61FCE019D
:1068B0000E940718813049F492E090938D058093EF
:1068C000820583E180934003D9CF8230B9F684E01A
:1068D00080938D0581E08093820583E1809340035E
:1068E000CDCF0E942652FC0146815781608571857B
:1068F00040938505509386056093870570938805BE
:1069000080E1809340030E94C61F62E975E0CE01DA
:1069100085D480919305813049F482E080938D0580
:106920001092820583E180934003A8CF882321F051
:1069300086E080934003A2CF82E080934003CE01A3
:106940000E94AB5441E150E0BE0186E995E00E940F
:10695000555B0E9496526093890570938A058093D7
:106960008B0590938C05BDD60E94A21C87CF80E139
:10697000809340030E94C61FCE018DD2909395054F
:10698000809394050296029750F482E080938D05DF
:1069900081E08093820583E1809340036FCF41E1E2
:1069A00050E0BE0186E995E00E94555BCE0129D2F8
:1069B0000E94A21C87E18093400360CF8091400336
:1069C00090E0FC013297E731F10508F061C0EF5526
:1069D000FF4F0C94C65980913F038F5F80933F0314
:1069E0008530D8F455C080913F038F5F80933F037B
:1069F000893198F408950E94320A90913F038130C2
:106A000039F4943609F444C084E680933F033EC0D1
:106A10009F5F90933F039530D8F110923F0336C0AB
:106A200080918E05813051F40E942F0AFC018081F3
:106A3000882321F083E08093400328C080918E0555
:106A4000823031F50E94E10B882311F188E18093B7
:106A500040030E94251CFC01148215820E94C61F5F
:106A60000C94A10A089580918F05882379F080E025
:106A70000E94FA15882311F080E006C081E00E9490
:106A8000FA15882319F081E00E94372C0C94C61F58
:106A90000895843508F083E5443508F043E5603314
:106AA00008F06FE2203308F02FE2E091A607F091A2
:106AB000A7079081891708F480838281841708F4DE
:106AC00042838181681708F461838381821708F407
:106AD00023830895E091A607F091A70783E58083BB
:106AE00012828FE281831382089548EF51E060E0C3
:106AF00070E08091A4079091A5070E94285B2FE287
:106B000043E560E080E0C5DF17C1089548EF51E03C
:106B100060E070E08091A4079091A5070E94285B37
:106B20002FE243E560E080E0B4CF08959093A5079D
:106B30008093A4077093A7076093A60708952AB5CA
:106B40003BB58091730590917405820F931F9BBD97
:106B50008ABD849B02C081E001C08FEF0E94075371
:106B60008091A8079091A907A091AA07B091AB07BF
:106B70000196A11DB11D8093A8079093A907A0932A
:106B8000AA07B093AB070895A2E0B0E0EAECF5E302
:106B90000C94715A89839A830E944B0989819A8146
:106BA0000E94E154082F8823A1F11CE280E00E949A
:106BB00007531150D9F70E940D531092A807109255
:106BC000A9071092AA071092AB071FBC20910501DC
:106BD0003091060140E050E060E074E284EF90E024
:106BE0000E94885930937405209373051DBC1CBC0A
:106BF00020917305309174053BBD2ABD2FE935E323
:106C0000309377052093760597B7906197BF81E021
:106C10008EBD802F2296E4E00C948D5A87B78F7E2C
:106C200087BF0E9491510E940D5360E070E0CB013C
:106C30000E94965362E579E486E496E40E94B406E5
:106C40006091A8077091A9078091AA079091AB075E
:106C50006C5D7F4F8F4F9F4F0E94B40667E571E4D4
:106C600086E595E40E94B40666E67DE684E790E258
:106C70000E94B40660E170E080E090E00E94B406FB
:106C800081E090E00E94AE0681E090E00E94AE06B6
:106C9000609105017091060180E090E00E94B406C9
:106CA000609105017091060180E090E00E94B406B9
:106CB00081E090E00E94AE0688E090E00E94AE067F
:106CC00064E671E684E791E60E94B4066091A80745
:106CD0007091A9078091AA079091AB070E94B40612
:106CE0000E940D530E94615381E008950F93909389
:106CF00069058093680560936A0540936B0520934E
:106D00006C0500936D0510926E050F910895C4985F
:106D10000C940F1C0895C49A0C940F1C0895CF93E3
:106D2000C82F81E2F4DF8C2F8068F1DF80E2EFDF93
:106D30008CE0EDDFCF910895EF92FF920F931F93B8
:106D4000CF93DF93C0E0D0E080E090E0E12CE091D1
:106D5000A607F091A7078C01085F1F4F218130E043
:106D6000201731073CF0E394CC5ADF4F0033110574
:106D700081F505C0238130E02817390734F4AADEF5
:106D8000CDB7DEB7E6E00C948B5A8E2D8064BFDF62
:106D9000E091A607F091A70780818068B8DFE091B5
:106DA000A607F091A707F080E091A607F091A7074A
:106DB00082818F15C0F20E94110AE091A407F09120
:106DC000A507EC0FFD1FEF0DF11D8081A4DFF394EB
:106DD000EBCFC801BCCF0E94181C81E298DF82E192
:106DE00096DF80ED94DF80E292DF8CE090CF089513
:106DF00087B78F7E87BF109284001B980C946153D5
:106E00000895CF92DF92EF92FF920E94AB548823B5
:106E1000C1F10E9436570E949C0662347745814436
:106E2000964519F0E5DF82E02DC00E9492060E948F
:106E300092061FBC1DBC1CBC6C01E12CF12CA0EE09
:106E4000BFEFA70196010E94E7597C5D8B409F4FE1
:106E50000E9488593BBD2ABD8AB59BB58FEF97E04C
:106E600090937705809376051092AD0791E090930B
:106E7000BC071092AC0787B7806187BF9EBD80E0DA
:106E800001C081E0FF90EF90DF90CF90089587B729
:106E90008295817008954F925F926F927F928F9248
:106EA0009F92AF92BF92CF92DF92EF92FF921F9389
:106EB000CF93DF93A8950E94AB54882309F4BFC0F9
:106EC0000E949C06623477458144964509F0B2C021
:106ED0000E949206029708F0ADC00E949206EC0153
:106EE000C13583ECD80708F0A5C061E070E080E010
:106EF00090E00E94C353882309F49CC00E94245749
:106F0000811132C081E08093BD0768E070E080E0CD
:106F100090E00E949653882309F48CC0C12CD12C98
:106F20007601A8950E942457882331F08F77C80EE8
:106F3000D11CE11CF11CF5CF0E9461539E0140E081
:106F400050E0C701B6010E94885969017A01CA015F
:106F5000B9012EEB30E040E050E00E9488592C0D42
:106F60003D1D4E1D5F1D64C08093BD079CE0899F41
:106F7000B00111246F5F7F4F882777FD8095982F90
:106F80000E94C353882309F455C010E0C12CD12CB2
:106F900076019AE0492E512C612C712C8091BD070D
:106FA000181730F50E949C060E949C060E949C06C1
:106FB0004B015C012EEB30E040E050E00E9488592C
:106FC000280D391D4A1D5B1DC20ED31EE41EF51E81
:106FD000C12FD0E0CC0FDD1FC85AD54FCA01B9016F
:106FE000A30192010E948859398328831F5FD6CF5D
:106FF0008091580A9091590AA0E0B0E08093AE07C2
:107000009093AF07A093B007B093B1078091AE07FC
:107010009091AF07A091B007B091B1070E94615362
:10702000C701B60128EE33E040E050E00E948859E5
:10703000C90107C00E9461538FEF9FEF02C08EEF1E
:107040009FEFDF91CF911F91FF90EF90DF90CF9056
:10705000BF90AF909F908F907F906F905F904F9078
:107060000895CF932091BD0730E0281B31092F5F91
:107070003F4F8CE0829FB001839F700D11246F5FA2
:107080007F4F80E090E00E94C353811102C0C0E0B6
:1070900009C00E949C060E949653C82F8823B9F30A
:1070A0000E94BF528C2FCF91089587B78F7E87BFE4
:1070B000109284001B9881E08093AC070895809122
:1070C000BC07CFDF882329F097B7906197BF109254
:1070D000AC070895CF92DF92EF92FF921F93CF9368
:1070E000DF936091BD078CE0689FB00111246F5F52
:1070F0007F4F882777FD8095982F0E94C353182FC4
:10710000882309F44AC0C1E0C12CD12C76018091BA
:10711000BC078C17D8F00E949C060E949C060E9417
:107120009C062091BC076C0D7D1D8E1D9F1DC217F6
:1071300018F46B017C0108C06093AE077093AF0731
:107140008093B0079093B107CF5FE1CFC701B6013D
:1071500028EE33E040E050E00E948859E9010E94A7
:10716000251CFC01CE016CE370E00E946159C82F20
:1071700064830E94251CFC01C5830E94251CEC0130
:107180000E94251CFC01848188830E94251CEC013F
:107190000E94251CFC0185818983812FDF91CF917D
:1071A0001F91FF90EF90DF90CF9008952091AC0752
:1071B000211133C04091AE075091AF076091B007E5
:1071C0007091B107A0E0B0E084179507A607B70754
:1071D00020F1E091BC078091BD07E817F0F4EF5F64
:1071E000E093BC078091AE079091AF07A091B007E4
:1071F000B091B107F0E0EE0FFF1FEA5AF54F208182
:107200003181820F931FA11DB11D8093AE07909312
:10721000AF07A093B007B093B1070895A0E0B0E026
:10722000E4E1F9E30C94635AEB011982188210929D
:10723000BD0710929505109294050E94AB548823C7
:1072400039F0C12CD12C7601412C512C32015BC07C
:1072500081E08983D0C00E942457B82E0E94245711
:10726000082F22E0420E511C611C711C882309F476
:1072700053C00E949652641575058605970508F45B
:107280004DC0A89510E0102F00270B0D111D0E9476
:1072900096524801A12CB12C6419750986099709E9
:1072A000681579058A059B05D8F18091BD078F5F28
:1072B0008093BD0753014201312C01501109C401D3
:1072C000841995098017910798F40E942457282E55
:1072D0003FEF831A930AA30AB30A0E9496526815D5
:1072E00079058A059B05F8F40E94965242E049838D
:1072F0000E942457240135012FEF421A520A620AD4
:10730000720A381223C00E94965246165706680623
:10731000790608F4A0CF23C0B110ABCF0E949652DB
:1073200082E089831CC0322488E027FC06C05FEF1E
:10733000C51AD50AE50AF50A05C092E0C90ED11CA6
:10734000E11CF11C220C815081F7B9CF8881811199
:10735000DACF33E039838091BD078883D4CF0E9490
:107360005A13EC010E9450138C010E946E135C01B1
:107370000E9478136091BD079C012A0D3B1DC00F30
:10738000D11F48EE53E0C49FC001C59F900DD49F0C
:10739000900D1124280F391F629F4001639F900CAC
:1073A0001124A12CB12C0E948213A7019601220F57
:1073B000331F441F551FDC010E94DB59860E971EA8
:1073C000A81EB91E0E940413A501940104C056957D
:1073D0004795379527958A95D2F7CA01B90120E4D8
:1073E00032E44FE050E00E94885930939505209395
:1073F00094050E946153CDB7DEB7E2E10C947F5A49
:10740000A0E0B0E0E6E0FAE30C946E5AD62E0E94BB
:10741000AB54E82E882309F44FC00E94F953109210
:10742000B2071092B3071092B4071092B507F12C6F
:10743000FD1409F441C00E94B952182F0E94B9529C
:107440004091B2075091B3076091B4077091B507AE
:107450004E5F5F4F6F4F7F4F4093B2075093B3071C
:107460006093B4077093B507C82FD0E0DC2FCC270A
:10747000C10FD11D00E010E00C171D07D9F00E94CC
:10748000B9524091B2075091B3076091B40770911F
:10749000B5074F5F5F4F6F4F7F4F4093B2075093D9
:1074A000B3076093B4077093B5070E94F9530F5F59
:1074B0001F4FE2CFF394BCCF8E2DCDB7DEB7E7E000
:1074C0000C948A5AA0E0B0E0E8E6FAE30C946D5A16
:1074D0008091B7079091B807A091B907B091BA070A
:1074E000892B8A2B8B2B09F4D9C08091C10784305A
:1074F00029F08091C107873009F0D0C08091BC0786
:1075000081116BC084E08093C1070E94B952C82FDB
:107510000E94B9524091B2075091B3076091B407ED
:107520007091B5074E5F5F4F6F4F7F4F4093B2072B
:107530005093B3076093B4077093B507282F30E0DA
:10754000322F22272C0F311D4091B7075091B807D9
:107550006091B9077091BA07C9010296481B590B8F
:10756000610971094093B7075093B8076093B90751
:107570007093BA078091BC078F5F8093BC0783B775
:10758000846083BF12BE87B7816087BF3093C00716
:107590002093BF070E9450138C010E946413EC01DA
:1075A0000E940413F82E9801A8EEB3E00E94CC5973
:1075B0009E0140E050E00E94AA590F2C04C056954D
:1075C0004795379527950A94D2F73093C5072093AE
:1075D000C4071092C10712BE7FC08091C1078730D7
:1075E00009F490CF0E945A13EC010E9404139E01EB
:1075F00002C0369527958A95E2F7C9016AE070E0E6
:107600000E9461597B010E94251CEC014C813D8147
:107610002E8180E797E1489F8001499F100D11243A
:1076200054E6359F000D111D1124020F111D2E81EE
:10763000F0E7CF2EF7E1DF2E5C814D813E815C9D2E
:10764000C0015D9D900D112454E6459F800D911D54
:107650001124830F911D801B910B8E159F0548F4FB
:107660008E81821749F3A8950E947315A7D92E81A0
:10767000E3CF8091C107863079F18091C1078530D1
:1076800059F18091B7079091B807A091B907B091CF
:10769000BA07892B8A2B8B2BF9F034CF8091B7074F
:1076A0009091B807A091B907B091BA07892B8A2B9E
:1076B0008B2B91F48091C107843021F08091C10718
:1076C000873051F40E9461530E942113811110925E
:1076D000840085E08093C107CDB7DEB7E8E00C9465
:1076E000895ACF931092BC0784E08093C10710920F
:1076F000B2071092B3071092B4071092B5070E9418
:1077000096526093B7077093B8078093B907909328
:10771000BA070E940413C82F0E9464139695879598
:10772000969587950C2E02C0969587950A94E2F758
:10773000282F20952093C2070E946E139695879557
:10774000969587950C2E02C0969587950A94E2F738
:10775000282F20952093C3070E947813969587952C
:10776000969587950C2E02C0969587950A94E2F718
:10777000282F20952093BE070E9482139695879507
:1077800096958795AC010C2E02C0569547950A94A4
:10779000E2F740954093B6079C01220F331F02C0C9
:1077A00036952795CA95E2F720952093C607CF9185
:1077B000089585E08093C1071092B7071092B8072B
:1077C0001092B9071092BA070E94211381111092EA
:1077D00084001092BB070C946153089586E0809357
:1077E000C1070E9421138111109284001092BB07DF
:1077F0000895A0E2B0E0EFEFFBE30C94715A0E9411
:107800009156BC01CE0101960E944E5B0E946153CD
:107810008091BC07882329F08091BC078150809318
:10782000BC076091BC07CE010196EADD0E9496522A
:107830000091B2071091B3072091B4073091B507BA
:10784000601B710B820B930B6093B7077093B807A3
:107850008093B9079093BA0787E08093C107A096F9
:10786000E4E00C948D5A6091B2077091B307809157
:10787000B4079091B50708959091C10781E09630C3
:1078800009F080E0089512BE8091C107843010F0A5
:107890001B9808958091BB07882361F01B9A0E9472
:1078A0002113882321F08091070180938400109296
:1078B000BB0709C01B980E942113811110928400FC
:1078C00081E08093BB078091C107811115C0809131
:1078D000C20782BF8091C4079091C507892B51F0E0
:1078E0008091C4079091C50701979093C507809335
:1078F000C40702C081E008C08091C107813039F41B
:107900008091C30782BF82E08093C1070895809170
:10791000C107823081F48091BE0782BF83E08093EB
:10792000C10780E180934403109243031092420305
:107930001092410308958091C107833009F049C036
:1079400080914403803178F18091BF079091C00706
:1079500020914103309142032817390710F084E049
:10796000D3CF109244030E94B95280934303809175
:10797000B2079091B307A091B407B091B5070196F3
:10798000A11DB11D8093B2079093B307A093B407D4
:10799000B093B50780914103909142030196909373
:1079A0004203809341038091430387FF03C080918A
:1079B000C60702C08091B60782BF9091440390FF32
:1079C00005C080914303880F809343039F5F90938A
:1079D00044030895A4E0B0E0E0EFFCE30C94675AA0
:1079E0004C01CB01BA018114910409F476C06230D4
:1079F00071058105910508F470C0D401ED91FC91E9
:107A00002085608071802B3089F524E030E040E0F3
:107A100050E00E943C5AF401A284B384C484D5840B
:107A2000E684F784008911890E94D15AF4E0EF2E90
:107A3000F12C8E010F5F1F4FF3010995882309F484
:107A40004CC049815A816B817C814115510561058A
:107A5000710509F442C0DB01CA01805F9F4FAF4F3F
:107A6000BF404097A105B105A0F537C022E030E046
:107A700040E050E00E943C5AD4011A96AC901A970C
:107A80001B96BC901B971C96CC901C971D96DC9067
:107A90001D971E96EC901E971F96FC901F97509670
:107AA0000C91509751961C910E94D15AE2E0EE2E13
:107AB000F12C8E010F5F1F4FF3010995882369F0A8
:107AC00089819A81AC0160E070E001978F3E9F4F01
:107AD00020F4342F252FCB0104C030E020E080E0DB
:107AE00090E0632F722F2496EEE00C94835AA2E16B
:107AF000B0E0EDE7FDE30C94635A1C012A013B0161
:107B0000009709F4F6C0423051056105710508F48B
:107B1000F0C0D1011A96BC91BD83F101F385FE83BB
:107B2000D1011C96BC91BF83F101F585F887D10185
:107B30001E96BC91B987F101F785FA87D10150965D
:107B4000BC91BB87F101F189FC87D101ED91FC91DA
:107B500080858B3009F0A5C0C301B20124E030E07C
:107B600040E050E00E943C5AAD80BE80CF80D88477
:107B7000E984FA840B851C850E94D15A2D873E87A3
:107B80006A016F87788B898B9A8BD101ED91FC917B
:107B90000190F081E02D04E0E02EF12C8E010F5FCA
:107BA0001F4F0995882309F4A4C089809A80AB806F
:107BB000BC8081149104A104B10409F498C0D501DA
:107BC000C401805F9F4FAF4FBF400897A105B1052B
:107BD00008F48FC0D501C401885F9F4FAF4FBF40ED
:107BE0000897A105B10518F4812C912C5401F101DD
:107BF00086A597A5A0A9B1A9892B8A2B8B2B21F447
:107C000046A657A660AA71AA19821A821B821C82F4
:107C1000D101ED91FC910480F581E02D14E0E12E7D
:107C2000F12C8E010F5F1F4F2D853E85A6016F85BC
:107C3000788989899A89099581149104A104B104EC
:107C400009F455C02401350187CF49805A80411479
:107C5000510409F44CC0C2014096089708F449C089
:107C6000B8EF4B16BFEF5B0610F0412C512C1A8277
:107C70001982D101ED91FC910480F581E02DA2E003
:107C8000EA2EF12C8E010F5F1F4F9301A401B50165
:107C9000C6010995612C712C4114510461047104D1
:107CA00031F1C301B20122E030E040E050E00E9437
:107CB0003C5AAD80BE80CF80D884E984FA840B859D
:107CC0001C850E94D15A39014A015B016C01D10126
:107CD000ED91FC910190F081E02DB2E0EB2EF12CC2
:107CE0008E010F5F1F4F09958111AFCF02C081E058
:107CF00001C080E06296E2E10C947F5AA9E2B0E014
:107D0000E4E8FEE30C94635A4C014CA35DA36EA31C
:107D10007FA30B871C872D873E87009709F42FC10F
:107D2000DC01ED91FC9111972081318139A728A7C1
:107D3000448155815A8B498B1A965C911A975B8BBB
:107D40001B968C911B978C8B1C969C911C979D8BE2
:107D50001D96AC91AE8BD4011E96BC91BF8BD40105
:107D60001F96BC91B88FD4015096BC91B98FD401A5
:107D70005196BC91BA8FD4019E964D905D906D90B6
:107D80007C90D197B1E0BBA32085F40182899389CF
:107D9000A489B5892B3041F01BA29C01AD015695F9
:107DA00047953795279509C09C01AD0192E05695FE
:107DB0004795379527959A95D1F72B8F3C8F4D8F07
:107DC0005E8FD4019E961D921D921D921C92D1979A
:107DD0002B8D3C8D4D8D5E8D2F8F38A349A35AA3DB
:107DE0001F82188619861A868F8D98A1A9A1BAA11B
:107DF000892B8A2B8B2B09F461C032E04316510486
:107E00006104710448F08B8D9C8DAD8DBE8D48163C
:107E100059066A067B0628F082E0482E512C612C18
:107E2000712C9BA1992329F1C301B20124E030E018
:107E300040E050E00E943C5AAB88BC88CD88DE8888
:107E4000EF88F88C098D1A8D0E94D15A19014F873D
:107E5000588BD62EC72EB82EA92E04E0E02EF12C7A
:107E60008E010F5F1F4FE8A5F9A50995811191C0FB
:107E700086C0C301B20122E030E040E050E00E9441
:107E80003C5AAB88BC88CD88DE88EF88F88C098D99
:107E90001A8D0E94D15A19014F87588BD62EC72EA2
:107EA000B82EA92E12E0E12EF12C8E010B5F1F4F90
:107EB000E8A5F9A509958111BBC061C02B853C855A
:107EC0004D855E85232B242B252B09F052C08CA1D8
:107ED0009DA1AEA1BFA10297A105B10508F454C0B0
:107EE0009BA1992319F12F81388549855A852983CA
:107EF0003A834B835C836CA17DA18EA19FA124E07A
:107F000030E040E050E00E943C5AAB88BC88CD880D
:107F1000DE88EF88F88C098D1A8D0E94D15AF4E022
:107F2000EF2EF12C8E010F5F1F4F1EC02F81388561
:107F30003E832D836CA17DA18EA19FA122E030E024
:107F400040E050E00E943C5AAB88BC88CD88DE8877
:107F5000EF88F88C098D1A8D0E94D15AE2E0EE2E3E
:107F6000F12C8E010B5F1F4FE989FA890995811168
:107F70000BC04F81588569857A85C401B8DD60E002
:107F800070E080E090E092C06F81788589859A8565
:107F90008DC089819A81AB81BC81892B8A2B8B2BE7
:107FA00009F05AC02B853C854D855E85232B242BFB
:107FB000252B09F449C02F81388549855A85232B03
:107FC000242B252B49F48FEF9FEFAFEFBFE0898380
:107FD0009A83AB83BC8308C02F81388549855A8535
:107FE00029833A834B835C83B4E0EB2EF12C8E0122
:107FF0000F5F1F4F91014F8558896D2D7C2D8B2D63
:108000009A2DE989FA890995882309F4B2CF2B853D
:108010003C854D855E8521503109410951092B87E9
:108020003C874D875E874F82588669867A8614C062
:108030008D819E81892B81F48B859C85AD85BE8544
:10804000892B8A2B8B2BD1F4D4019E964D925D9275
:108050006D927C92D1973BCF2F8D38A149A15AA127
:1080600021503109410951092F8F38A349A35AA33F
:108070003FEF431A530A630A730AB6CE2F8138853D
:1080800049855A85232B242B252B29F44FEF5FEFAD
:108090005E834D8304C08F8198859E838D83A2E08B
:1080A000EA2EF12C8E010B5F1F4FA4CFA996E2E1BF
:1080B0000C947F5A80E190E00895A0E0B0E0E3E600
:1080C000F0E40C946B5AEC010097E1F0423051055A
:1080D00061057105B8F0CB01BA01625071098109DF
:1080E0009109288D398D40E050E00E943C5AAA8CBD
:1080F000BB8CCC8CDD8CEE8CFF8C08A119A10E946E
:10810000D15A08C020E030E040E050E060E070E08C
:1081100080E090E0CDB7DEB7EAE00C94875AFC012E
:10812000819191E080FB879587F92191820F9F5F74
:108130009B30C1F70895A0E0B0E0E1EAF0E40C94D0
:108140006D5A8C01F701C480D580C0E0D0E0C80131
:108150008C0F9D1FCC15DD0598F40E949C51892B36
:1081600069F4F70140815181628173814F5F5F4FF4
:108170006F4F7F4F40835183628373832296E7CF93
:1081800081E0CDB7DEB7E8E00C94895AADE0B0E00D
:10819000ECECF0E40C94655A6C0149012A013B01B6
:1081A000D701AD90BC90119712968D919C91139729
:1081B000809613969C938E931297F6018081853E4C
:1081C00011F0811104C0D70114961C924FC0F60122
:1081D00083858F3009F04CC0D70114968C91882389
:1081E00019F095858917A9F045E350E060E070E04B
:1081F000C5010E94285BF6018585D70114968C93F2
:10820000F50105A716A787A690AA41AA52AA63AAB4
:1082100074AAD6018C918F7390E001974DE0489F2E
:108220009001499F300D1124E8E0F1E0DE01119644
:1082300001900D924A95E1F7FE013196A20EB31E10
:10824000AE01425F5F4F2E1B3F0BC9018E0F9F1F78
:108250004F9760F48191B601680F711DDB018C911D
:10826000D5018D935D01E417F50779F781E0A9C089
:10827000F5018081882341F0C60151DFD7011496B2
:108280009C91981709F459C045E350E060E070E014
:10829000C5010E94285BF50105A716A787A690AA2D
:1082A00041AA52AA63AA74AAD601A50180E09C91B2
:1082B000903299F0FA019083F601248523FF07C0DC
:1082C0002C9121542A3118F4905EFA0190838F5F2B
:1082D00011964F5F5F4F883051F7D5019C919530D3
:1082E00011F495EE9C93F6019085903211F1F50111
:1082F000E80FF11D9EE29083F601389634E0380FC6
:108300008F5F90819032A9F0A501480F511DDA01CD
:108310009C93D6011C962C9124FF07C020812154E8
:108320002A3118F4905EDA019C938F5F31968313A3
:10833000E8CFF501E80FF11D1082F6018385D50124
:1083400090968C93C6014A960E949C512C01612CF8
:10835000712CF50145A256A267A270A6C6014496EB
:108360000E949C51AC0160E070E0BA01552744279F
:108370004429552966297729D50195964D935D9312
:108380006D937C939897C6014C960E94A451F50179
:1083900061A772A783A794A7C60146960E949C5125
:1083A000D50192969C938E939197C60148960E9410
:1083B0009C51F50194A383A381E0D70115968C937A
:1083C00080E02D96E0E10C94815AA0E0B0E0EBEE65
:1083D000F1E40C946D5A8C01F701C480D580C0E0A3
:1083E000D0E0C8018C0F9D1FCC15DD05A8F40E94BC
:1083F000A451672B682B692B69F4F70140815181E7
:10840000628173814F5F5F4F6F4F7F4F4083518316
:10841000628373832496E5CF81E0CDB7DEB7E8E0D1
:108420000C94895AAAE2B0E0E8E1F2E40C94635AB1
:108430006C014B01009711F480E089C16115710551
:10844000D9F3CE0181967C018E010E5D1F4F9E01F6
:108450002D5D3F4FAE014C5D5F4FBE016B5D7F4FA9
:1084600080970E947A1C29813A812C5B3740322FF9
:108470002227330F8DA1A0E28A9FC0011124282B4F
:10848000392B8CA1282BF40134A323A32AA1F0E2D9
:108490002F9F900111248BA190E0982F8827990F8E
:1084A000990F990F282B392B89A18695282BD40158
:1084B00092963C932E939197D601ED91FC918481F5
:1084C00095819AA789A7D4019D96BC91BEA3F4017A
:1084D000F6A5FFA3D4019F96BC91B8A7F40160A8AC
:1084E00051A842A833A824A8C4010E94695B6C016A
:1084F000182F99270C966DE070E00E947559762E22
:108500004BE050E060E270E0CE0101960E94285BF3
:108510006EE270E0C4010E948F5B0097C9F0DC013D
:1085200011962C912223A1F05C01BFEFAB1ABB0A7C
:10853000C5010E94695B1FEF1C0D181B482F84307A
:1085400008F043E050E0B501CE0109960E941F5BA0
:10855000193098F4412F50E0B401CE0101960E94E9
:108560001F5BF40180818E3211F581818E3209F416
:10857000828181111CC0712C1AC048E050E0B40106
:10858000CE0101960E941F5BD40195968C91982F85
:1085900092959F70803A10F4905D01C09F599F831F
:1085A0008F708A3010F4805D01C08F59888789816F
:1085B000853E11F485E0898345E150E060E070E09C
:1085C000CE010C960E94285BF40180A18C8761A1EA
:1085D00072A1CE0147960E94B351D40193966D913A
:1085E0007C919497CE0149960E94B351F40185A1E4
:1085F00096A1A7A1B0A5BD0188279927CE014596D0
:108600000E94B351D40195966D917C919697CE01BD
:108610004B960E94B351F40141A552A563A574A5E0
:10862000CE014D960E94B751F0E27F9EA001112429
:108630009A0140E050E060E070E080E090E0AEA0A1
:10864000BFA0C8A4D62CE52CF42C032D122D0E941B
:10865000D15A00E2E02EF12C8E010F5F1F4FE9A5E9
:10866000FAA50995882309F4E7CEC80158DDC82E7C
:10867000D72CADE0BA2EBFE0AB2EDD2009F461C0EF
:1086800040E250E06FEF70E0CE0101960E94285B5F
:108690008D2D90E00197B89EF001B99EF00D112448
:1086A000E80DF91D81E021E0280F9191A1E0B0E0F3
:1086B000AC0FBD1FA80FB11D9C938E5FA1E0B0E071
:1086C000AC0FBD1FA20FB11D1C928B3019F08A3167
:1086D000D1F102C08EE038C0992311F08F3118F328
:1086E000D982D71003C08D2D80648983AC86CE8655
:1086F0001D861B8E1C8EF0E2EF2EF12C8E010F5F7B
:108700001F4F2EA13FA148A5562D652D742D832DF9
:10871000922DE9A5FAA509952EA13FA148A5562DB0
:10872000652D742D832D922DA0E20E94DA5A2EA37E
:108730003FA348A7652E562E472E382E292EDA94B1
:108740009CCF81E004C08CE19111ADCFC9CFAA9636
:10875000E2E10C947F5AA2E1B0E0E1EBF3E40C9487
:10876000655A8C01423051056105710548F1A5DC5F
:108770002A013B014C0140E150E060E070E0CE0195
:108780000196298B3A8B0E94285BD801ED91FC91D0
:1087900011975896ED90FC9059970680F781E02D3F
:1087A000A12CB12C5AE5C52E50E4D52E8E010F5FB9
:1087B0001F4F29893A89A201B301C401099501C05B
:1087C00080E06296E0E10C94815AA0E2B0E0EBEE2A
:1087D000F3E40C94635A1C014B01CA0121143104C7
:1087E00009F470C1009709F46DC10E94695B0C9691
:1087F0006DE070E00E9461596F5F68A3D4014D90F5
:108800005D906D907C90D101ED91FC9111978085E8
:108810004114510461047104E9F58B3039F49A96DE
:108820004D905D906D907C909D9734C0F101F2A1C8
:10883000FA83D1019396BC91BB83F101F4A1FC832F
:10884000D1019596BC91BD83F101F6A1FE83D101C2
:108850009796BC91BF83F10180A491A4F28DF88F0B
:10886000D1015B96BC91B98FF101F48DFA8FD101E2
:108870005D96BC91BB8FF101F68DFC8FD1015F96A7
:10888000BC91BD8FF101F0A1FE8FD1019196BC91F9
:10889000BF8F10C0188E198E1A8E1B8E1C8E1D8EC7
:1088A0001E8E1F8E1A821B821C821D821E821F82B8
:1088B000812C912CEA81E88BFB81F98B0C810A8B4E
:1088C0001D811B8B2E812C8B3F813D8B8E8A9F8A35
:1088D00018862A813B814C815D816E817F81C40134
:1088E000A88CB98CCA8CDB8CEC8CFD8C0E8D1F8D0A
:1088F0000E94EF5A09F08FC04114510461047104C1
:1089000009F4E0C0A0E00E94F85A09F440C0B301A5
:10891000A201C1015FD86115710581059105A9F515
:1089200001E010E020E030E0B301A201C101E6D98E
:108930002B013C01611571058105910509F4C2C047
:108940006250710981099109D10158962D913C918C
:10895000599740E050E00E943C5AF101A28CB38C40
:10896000C48CD58CE68CF78C00A111A10E94D15A41
:10897000288B398B4A8B5B8B6C8B7D8B8E8B9F8B83
:10898000B301A201C101E7DE94C02B013C01B30198
:10899000A201C10192DB2A833B834C835D836E83FA
:1089A0007F834C01D10158968D919C9159978C01F0
:1089B00020E030E040E050E0BA0119872A873B8789
:1089C0004C875D876E877F872A813B814C815D81E3
:1089D0006E817F81C4015801C12CD12CE12CF12C76
:1089E00000E010E00E94D15A288F398F4A8F5B8FA8
:1089F0006C8F7D8F8E8F9F8F1A81188B2B81298B87
:108A00003C813A8B4D814B8B5E815C8B6F816D8B92
:108A10008E8A9F8A1886D101ED91FC910190F08198
:108A2000E02DEE24E394F12C8E010F5F1F4F2A817D
:108A30003B814C815D816E817F81C40109958823D2
:108A400009F440C08981853E11F0811118C0B885B4
:108A5000BF5FB887E8A1BE1760F52A813B814C81D2
:108A60005D816E817F81C401A0E20E94DA5A2A836F
:108A70003B834C835D836E837F834C012ACF2A81A5
:108A80003B814C815D816E817F81C401A0E20E94A7
:108A9000DA5A288B398B4A8B5B8B6C8B7D8B8E8B58
:108AA0009F8B2A833B834C835D836E837F834C0142
:108AB0000FCF288939894A895B896C897D898E899C
:108AC0009F8908C020E030E040E050E060E070E0C6
:108AD00080E090E0A096E2E10C947F5AA9E4B0E037
:108AE000E4E7F5E40C94635A9FA38EA3009709F47E
:108AF00022C2DC0114968D919C911597892B09F463
:108B00001AC216968D919C911797892B09F413C25E
:108B10008091FC049091FD04892B09F00CC242E382
:108B200050E060E070E08CEF94E00E94285B0EA1C2
:108B30001FA11093FD040093FC04D80119966D91B8
:108B40007D918D919C911C9720E032E040E050E0B7
:108B50000E943C5A322E232E6A0168AB79AB8AAB55
:108B60009BABABE00E94DA5AD801ED91FC91A5E2F3
:108B7000EA2EF12C8E010F5F1F4F0995811105C060
:108B80001092FD041092FC04D6C1CE0101960E9401
:108B90009C519FA78EA7CE0104960E949C518C01E8
:108BA000BB81BEAFEE81EFAFCE0107960E949C5114
:108BB00022969FAF8EAF2297CE0109960E949C51BC
:108BC0003C01CE010C960E949C5199AF88AFCE011A
:108BD00046960E94A4514B015C01CE014A960E9428
:108BE000A4516CAB7DAB8EAB9FABCE0182960E9445
:108BF000A4512A966CAF7DAF8EAF9FAF2A97811498
:108C00009104A104B10439F46114710409F4B8CFDA
:108C10004301A12CB12CE8ACF9ACE114F10441F012
:108C2000C701A0E0B0E08CAB9DABAEABBFAB09C061
:108C30008CA99DA9AEA9BFA9892B8A2B8B2B09F4DE
:108C40009FCF24013501401A510A610871089FAD78
:108C5000892F90E0A0E0B0E026968CAF9DAFAEAF3C
:108C6000BFAF26972CA93DA94EA95FA9BC01CD0194
:108C70000E944659461A570A680A790A8EA59FA586
:108C8000019722962EAD3FAD2297B5E0220F331FFC
:108C9000BA95E1F7820F931F6EA57FA50E946159D7
:108CA000461A570A61087108AEAD2A2F30E040E03D
:108CB00050E0C301B2010E9488592AAF3BAF4CAFCC
:108CC0005DAF253FBFE03B074105510508F458CF94
:108CD000253F3F4F4105510530F486E0AEA1BFA1CD
:108CE00018968C9304C08BE0EEA1FFA180874CE224
:108CF00050E060E070E08EEF94E00E94285BEEA40C
:108D0000FFA42701612C712CC501B401A3019201BC
:108D10000E943C5A2093FE043093FF0440930005C8
:108D20005093010560930205709303058093040539
:108D300090930505B80180E090E0A30192010E94A4
:108D40003C5AA32CB22CE8A8F9A80AA91BA90E9496
:108D5000D15A28AB39AB4AAB5BAB1B014C0120931A
:108D60000605309307054093080550930905609365
:108D70000A0530920B0580930C0590920D056AADA3
:108D80007BAD8CAD9DAD6E5F7F4F8F4F9F4FAEA182
:108D9000BFA118962C91263029F422E030E040E063
:108DA00050E004C024E030E040E050E00E9446592A
:108DB00060930E0570930F05809310059093110535
:108DC000EEA5FFA5F0931305E0931205AEACAE9EA1
:108DD000C001AF9E900D112490931505809314054A
:108DE000AEA1BFA118968C91863009F057C0E8ADAE
:108DF000F9AD9F0140E050E0C301B2010E943C5A2E
:108E0000AFACB12CC12CD12CE12CF12C00E010E046
:108E10000E94EB59A8A8B9A8CAA8DBA871018401CF
:108E20000E94D15A19012A013B014C0120931E05D1
:108E300030921F0540932005509221056093220532
:108E40007092230580932405909225052296AEAC5E
:108E5000BFAC2297B50180E090E020E230E040E036
:108E600050E00E943C5A59016A017B018C0191013A
:108E7000A201B301C4010E94D15A20931605309378
:108E80001705409318055093190560931A057093C0
:108E90001B0580931C0590931D054AC0CEA4DFA43A
:108EA000B60180E090E026962CAD3DAD4EAD5FADB5
:108EB00026970E943C5ACCA8DDA8EEA8FFA8560130
:108EC0006701E12CF12C8701AEA2BFA2C8A6D9A6EA
:108ED000EAA6FBA60CA71DA7E12CF12C00E010E0F0
:108EE0000E94EB59A8A8B9A8CAA8DBA871018401FF
:108EF0000E94D15A20931605309317054093180508
:108F00005093190560931A0570931B0580931C05F7
:108F100090931D052A96ECACFDAC0EAD1FAD2A97C3
:108F2000E0922605F0922705009328051093290565
:108F30008CEF94E002C080E090E0C75BDF4FE2E19D
:108F40000C947F5A009719F0FC0111821082089549
:108F5000EF92FF920F931F93CF93DF937C018B01CE
:108F6000009799F06115710581F0FB0180A184FDE6
:108F70000CC08091760490917704892B49F0809100
:108F8000B9049091BA04892B31F080E090E024C0BC
:108F9000C6E7D4E002C0C9EBD4E045E350E0B80135
:108FA000CE0102960E941F5BF982E8821FAA18AECA
:108FB00019AE1AAE1BAE1CAE1DAE1EAE9E01215CDC
:108FC0003F4FF80185A196A1A7A1B0A5F901808323
:108FD0009183A283B383CE01CDB7DEB7E6E00C94D4
:108FE0008B5ACF93DF93EC01009741F0BC016E5F89
:108FF0007F4F8881998116DA19821882DF91CF918B
:109000000895ACE1B0E0E7E0F8E40C94635A9A8F7D
:10901000898F7E8B6D8B5A8B498BDC01D796BC91E7
:10902000B983FC01F0ADFA83DC01D996BC91BB8316
:10903000FC01F2ADFC83DC01DB96BC91BD83FC013D
:10904000F4ADFE83DC01DD96BC91BF83FC01F6AD7F
:10905000F887DC019B964D905D906D907C909E977B
:109060004A019A0140E050E060E070E080E090E06A
:10907000A980BA80CB80DC80ED80FE800F811885CE
:109080000E94D15A63015201E12CF12C87014986DB
:10909000BA86CB86DC86ED86FE860F87188BE12CA0
:1090A000F12C00E010E00E94EF5A41F038F062012C
:1090B000E980FA80CE18DF08DA8AC98A09891A8914
:1090C0000115110509F420C1A98DBA8DED91FC910E
:1090D0001197A08CB18CBC8AAB8AFD01FF964080B1
:1090E000518062807380411451046104710409F05D
:1090F00050C097964D905D906D907C909A974114DA
:10910000510461047104A9F4E1E0F0E029813A819D
:109110004B815C816D817E818F819885A0E00E946A
:10912000F85A11F4E0E0F0E0882799278E1B9F0B96
:10913000EDC029813A814B815C816D817E818F8177
:109140009885A0E00E94F85A21F1C980DA80EB806E
:10915000FC800B891C894801A12CB12CC814D904AE
:10916000EA04FB04B0F0C818D908EA08FB08B30108
:10917000A201A98DBA8D8D919C910E94EA3C2B0190
:109180003C01611571058105910541F78FEF9FEF56
:10919000BDC0EB89FC893197A980BA80EA21FB2107
:1091A000FA87E98729883A88098D1A8D015C1F4F53
:1091B0001A830983A98DBA8D0D911C91B301A20167
:1091C000C8010E945D4059016A017B018F8B988F15
:1091D0008B889C88E985FA858E1A9F0A28143904A1
:1091E00008F44101D8010D90BC91A02DBC8FAB8F2C
:1091F000E985FA859F0140E050E060E070E080E0A2
:1092000090E00F89188D0E94D15AAB8DBC8DED91E5
:10921000FC9174010D891E890995882309F460C0A9
:10922000ED89FE89E80DF91DFE8BED8B28183908B4
:10923000940140E050E060E070E080E090E0A98DB3
:10924000BA8DD796AC90D797D896BC90D897D99628
:10925000CC90D997DA96DC90DA97DB96EC90DB9796
:10926000DC96FC90DC97DD960C91DD97DE961C91E8
:10927000DE970E94D15AD7962C93D797D8963C93D5
:10928000D897D9964C93D997DA965C93DA97DB9670
:109290006C93DB97DC967C93DC97DD968C93DD9763
:1092A000DE969C93DE97E985FA858E0E9F1EAB882D
:1092B000BC888A149B04D8F0B301A2018D919C91C3
:1092C0000E94EA3C2B013C01611571058105910565
:1092D00061F4A981BA811D921D921D921C9213976F
:1092E00089899A898219930911C01A861986E98198
:1092F000FA8140825182628273822114310409F022
:1093000059CF89899A8902C080E090E06C96E2E1A9
:109310000C947F5AA4E1B0E0E0E9F9E40C94635ABC
:109320009C8B8B8B7C876B875E874D87892B19F491
:109330008FEF9FEFDCC12B853C85232BC9F38D85F7
:109340009E85892BA9F3AB89BC89D796BC91B9833B
:10935000EB89FC89F0ADFA83AB89BC89D996BC91C5
:10936000BB83EB89FC89F2ADFC83AB89BC89DB96BE
:10937000BC91BD83EB89FC89F4ADFE83AB89BC89CC
:10938000DD96BC91BF83EB89FC89F6ADF887EB894C
:10939000FC8983A594A5A5A5B6A51C012D01612C6A
:1093A000712C430129813A814B815C816D817E81E1
:1093B0008F81988551016201E12CF12C00E010E0D1
:1093C0000E94EF5A11F008F0B3CF0190F081E02D28
:1093D000208D318D3A872987AB89BC89DF964D90E6
:1093E0005D906D907C90190131E0231A31088981DC
:1093F0009A8128223922411451046104710409F030
:1094000081C0AB89BC8997964D905D906D907C90A2
:109410009A97411451046104710419F529813A8124
:109420008F819885A0E00E94F85A09F081CF01E071
:1094300010E020E030E040E050E0BA01CF010E94AF
:109440007E3E2B013C01EB89FC8967A370A781A7B5
:1094500092A7611571058105910519F480E090E0EE
:1094600046C1AB89BC89D7961C91D797D896BC9139
:10947000EB89FC8901ADF2AC63AD74AD212F3B2FBC
:10948000402F5F2D85AD96ADA0E00E94F85AD1F136
:10949000812E9B2EA02EBF2C29853A856901E12CB7
:1094A000F12C8C149D04AE04BF0460F18C189D084F
:1094B000AE08BF08B301A201AB89BC898D919C9114
:1094C0000E94EA3C6115710581059105C1F4811482
:1094D0009104A104B10409F02BCF01E010E020E0D9
:1094E00030E0B301A201EB89FC89808191810E9467
:1094F0007E3E611571058105910509F4AFCF2B0101
:109500003C01CFCF2D853E853A8329838B899C8969
:10951000CF969A8B898BAB89BC890D90BC91A02D7D
:10952000B88BAF87B301A201CD010E945D40590104
:109530006A017B018C0189849A8482189308E981ED
:10954000FA81E815F90508F44F01AF85B889ED9166
:10955000FC91910140E050E060E070E080E090E03C
:109560000E94D15A0480F581E02D74010B851C8581
:109570000995882309F489C0EB85FC85E80DF91D60
:10958000FC87EB8729813A81281939093A83298395
:10959000940140E050E060E070E080E090E0AB8952
:1095A000BC89D796AC90D797D896BC90D897D996C7
:1095B000CC90D997DA96DC90DA97DB96EC90DB9733
:1095C000DC96FC90DC97DD960C91DD97DE961C9185
:1095D000DE970E94D15AD7962C93D797D8963C9372
:1095E000D897D9964C93D997DA965C93DA97DB960D
:1095F0006C93DB97DC967C93DC97DD968C93DD9700
:10960000DE969C93DE97820C931CE985FA858E1674
:109610009F0678F1B301A2018D919C910E94EA3CD2
:10962000611571058105910501F529813A81232B89
:1096300041F4A989BA891D921D921D921C9213971B
:1096400024C001E010E020E030E0B301A201EB898A
:10965000FC89808191810E947E3E2B013C01611535
:1096600071058105910519F4E4CF2B013C01212CF2
:10967000312CA989BA894D925D926D927C92139793
:10968000E981FA81EF2B09F046CFEB89FC89B7A974
:10969000A0ADF1ADF987EB89FC89F2ADFB87EB89D1
:1096A000FC8963AD74AD03A514A525A536A51801E5
:1096B0002901612C712C43012B2F3A2F49855B85A1
:1096C00085AD96AD51016201E12CF12C00E010E076
:1096D0000E94EF5A31F028F09D0133A724A745A737
:1096E00056A78D859E8529813A81821B930B6496AE
:1096F000E2E10C947F5AA0E1B0E0E1E8FBE40C94D5
:10970000635A4C012A013B01009711F480E097C194
:10971000DC019796CD90DD90ED90FC909A97ED91BD
:10972000FC91808D918DC114D104E104F10461F0AC
:109730004D825E826F8278868C0120E030E00D875A
:109740001E872F87388B24C041155105610571058F
:1097500079F724C1B701A601D4018D919C910E9493
:10976000EA3C611571058105910521F1ED80FE80CE
:109770000F8118852D853E854F855889E21AF30A99
:10978000040B150BED82FE820F8318876B017C01A1
:109790004D815E816F8178858D859E85AF85B88985
:1097A00084179507A607B707A8F2C114D104E104EE
:1097B000F10489F56D857E858F8598890D811E81DF
:1097C0002F813885600F711F821F931F61507109AF
:1097D000810991092D853E854F8558890E948859B8
:1097E00089019A01B701A601D4018D919C910E9433
:1097F0007E3E611571058105910509F487CFC1147D
:10980000D104E104F10439F4F40167A370A781A73E
:1098100092A76B017C01D4019B964D925D926D9253
:109820007C929E97411451046104710429F4F4015F
:1098300017A210A611A612A6B4016E5F7F4FD40125
:109840008D919C910E941242882309F45FCF4114AC
:1098500051046104710431F4B701A601F40180815F
:1098600091819AC00D811E812F8138854D855E853D
:109870006F857889401751076207730708F48EC017
:10988000D4012D903C902114310409F487C0B2E03A
:10989000CB16D104E104F10408F480C0B701A6019D
:1098A000C1010E94EA3C6D837E838F839887D1013A
:1098B000ED91FC918085048115811E870D878B3089
:1098C00071F58FEF9FEFAFEFBFE089839A83AB8392
:1098D000BC83C701B60124E030E040E050E00E94C4
:1098E0003C5AD1011A96AC901A971B96BC901B97C4
:1098F0001C96CC901C971D96DC901D971E96EC90A4
:109900001E971F96FC901F9750960C91509751965A
:109910001C910E94D15A04E0E02EF12C29C08FEF57
:109920009FEF9A838983C701B60122E030E040E0CF
:1099300050E00E943C5AD1011A96AC901A971B969F
:10994000BC901B971C96CC901C971D96DC901D9785
:109950001E96EC901E971F96FC901F9750960C91A8
:10996000509751961C910E94D15A12E0E12EF12C91
:109970008E010F5F1F4FED85FE850995882371F0DD
:10998000ED80FE800F811885E114F10401051105B9
:1099900029F0B801A701C1010E94773D930182011E
:1099A00040E050E0BA014D821E832F8338874987FB
:1099B0005A876B877C87D401D796AC90D797D89677
:1099C000BC90D897D996CC90D997DA96DC90DA9754
:1099D000DB96EC90DB97DC96FC90DC97DD960C91A7
:1099E000DD97DE961C91DE972D813E814F81588553
:1099F00060E070E080E090E00E94EF5AF8F4D796C3
:109A00002C93D797D8963C93D897E42ED9964C931D
:109A1000D997F52EDA965C93DA97DB961C92DB9752
:109A2000DC961C92DC97DD961C92DD97DE961C92EC
:109A3000F401FF96108211821282138281E06096F7
:109A4000E2E10C947F5AA0E0B0E0E9E2FDE40C947E
:109A5000655AEC018B01009709F453C0611571053B
:109A600009F44FC06FA958AD39AD2AAD4130A1F00E
:109A700068F0423009F045C0F801408051806280B2
:109A800073808BA59CA5ADA5BEA50FC0F801408035
:109A90005180628073800DC0862F952FA32FB22F27
:109AA000F8014080518062807380480E591E6A1E02
:109AB0007B1E8BA59CA5ADA5BEA584159505A60509
:109AC000B705C8F053014201C12CD12C76014FAA31
:109AD00098AEA9AEBAAE1BAE1CAE1DAE1EAEEF96D2
:109AE000188219821A821B82F80140825182628296
:109AF000738281E007C0B301A201CE01FCDD8111B8
:109B0000E1CF80E0CDB7DEB7E0E10C94815AEF926F
:109B1000FF920F931F93CF93DF937C018B010097EC
:109B200091F06115710579F0FB0180A184FF0BC0F4
:109B3000C5E4D3E088819981892B41F0ED96F4E06A
:109B4000C637DF07B9F780E090E015C045E350E085
:109B5000B801CE0102960E941F5BF982E882F801EB
:109B600085A196A1A7A1B0A58FAB98AFA9AFBAAFB9
:109B70001CAE1BAECE01CDB7DEB7E6E00C948B5A1F
:109B8000009719F0FC01118210820895FC010097E2
:109B900061F047A150A561A572A547AB50AF61AF79
:109BA00072AF14AE13AE81E0089580E00895A6E38D
:109BB000B0E0EDEDFDE40C94635A9AA789A78B0100
:109BC000892B01F161157105E9F0A9A5BAA52D90C0
:109BD0003C901197F101008CF18DE02DFCA7EBA7D3
:109BE000D7964D905D906D907C90DA97DB962D9195
:109BF0003C91DC9738A72FA32E173F0728F089A5A3
:109C00009AA5C4DF80E0CCC046E050E060E070E0A0
:109C1000CE0181960E94285B45E350E060E070E051
:109C2000C8010E94285B1AA309A3411451046104CE
:109C3000710409F080C0D101ED91FC9111978085EC
:109C40008B3039F49A964D905D906D907C909D97F5
:109C500072C0F101028CF38DE02DD10192968D91AD
:109C60009C919397E81BF90BFCA7EBA764C0EBA5AD
:109C7000FCA52FA138A5E21BF30BFEABEDABA901B0
:109C800060E070E080E090E0DC012DA75EA76FA7A8
:109C900078AB89AB9AABABABBCAB4114510461045C
:109CA000710409F04DC040E050E060E070E080E0F9
:109CB00090E0D1019296AC9092979396BC90939736
:109CC0009496CC9094979596DC9095979696EC9078
:109CD00096979796FC90979798960C919897999647
:109CE0001C910E94D15A1CA21BA2D101ED91FC91A2
:109CF0000280F381E02DDE0191964D01A6ECAA2EA3
:109D0000A0E4BA2ECDA8DEA8B0E2EB2EF12C8E0195
:109D10000F5F1F4F0995882309F474CF8BA19CA175
:109D2000EFA1F8A5E80FF91FF8A7EFA32BA53CA515
:109D3000E217F30798F48EA1882309F498CF21C085
:109D4000B301A201C1010E945D40ADA4BEA4C12C1B
:109D5000D12CE12CF12C00E010E0C3CFB301A20123
:109D6000C1010E94EA3C2B013C016115710581058E
:109D7000910521F48EA1811104C041CF18A61FA224
:109D8000DACFA9A5BAA5D7964D925D926D927C9235
:109D9000DA97EFA1F8A5DC96FC93EE93DB978EA102
:109DA000E696E2E10C947F5AA0E0B0E0EAEDFEE432
:109DB0000C94695A5C01EB018A01009709F45EC0BA
:109DC000209709F45BC08881882309F457C04115A6
:109DD000510509F453C08F3209F4219645E350E050
:109DE00060E070E0C8010E94285B80E1F80180A378
:109DF0008881811102C081E042C0B801C50187DEBF
:109E00007C010097D9F16FE270E0CE010E943A5BCD
:109E1000009741F0C82ECC1A4C012FEF821A920AFB
:109E2000D12C0EC0CE010E94695BC82E4E01880E57
:109E3000911CF6CFC8010E94695B8C159D0531F01D
:109E4000B801C701B4DE8111F5CF15C0A601B80174
:109E5000CE010E94725B892B99F7C70191DECC0D70
:109E6000DD1D8881882339F2F80180A184FF06C0B6
:109E7000E401E12CF12CC70183DEBACF80E0CDB73D
:109E8000DEB7ECE00C94855AA0E0B0E0EAE4FFE431
:109E90000C946D5A8C017B01EA01009709F443C0D0
:109EA0006115710509F43FC0FB0180818823D9F158
:109EB0002097C9F1BE01C8017ADE882351F0BE01A6
:109EC000C7010E94455B892BA9F7C8015FDE92E0BC
:109ED0002BC0F801C080D18045E350E060E070E025
:109EE000CE010E94285B4FE150E0B701CE010E94F5
:109EF000805BB801695D7F4FAE01C6010E94E543FA
:109F00002DA73EA74FA758AB69AB7AAB8BAB9CABE9
:109F1000A0E00E94F85A39F0BE01C6010E94124228
:109F200091E0811101C090E0892FCDB7DEB7E8E064
:109F30000C94895AFC01009711F1A081B181189607
:109F40004C9182899389A489B589208D318DBC017A
:109F5000CD014B3041F4F2E0969587957795679562
:109F6000FA95D1F704C096958795779567956250D5
:109F700071098109910940E050E00C943C5A20E0BD
:109F800030E040E050E060E070E080E090E0089574
:109F9000A0E3B0E0EEECFFE40C94635A3C010097C0
:109FA00049F420E030E040E050E060E070E080E024
:109FB00090E091C019A21AA21BA21CA280E290E01C
:109FC0009EA38DA3F301F285F9A7F301F385FAA708
:109FD000F301F485FBA7F301F585FCA7F301F685F2
:109FE000FDA7F301F785FEA7F301F089FFA7F301B1
:109FF000F189F8ABF301228833884488558821140D
:10A0000031044104510409F45BC0FEEF2F16FFEF49
:10A010003F064104510418F438A62FA204C02EEFC5
:10A020003FEF38A72FA3A895F301A081B181129625
:10A03000ED91FC91139718968C91863019F48BE969
:10A0400090E402C085EE91E49E012F5D3F4F4901EF
:10A050005C01CFA0D8A4A0E2EA2EF12C8E010F5F04
:10A060001F4F29A53AA54BA55CA56DA57EA58FA57B
:10A0700098A90995882309F494CFCFA0D8A44601C4
:10A08000960140E050E060E070E080E090E0A9A43C
:10A09000BAA4CBA4DCA4EDA4FEA40FA518A90E9429
:10A0A000D15A29A73AA74BA75CA76DA77EA78FA770
:10A0B00098AB8FA198A5281A390A410851089FCF5B
:10A0C00069A17AA18BA19CA1F301208D318D40E083
:10A0D00050E00E943C5AE096E2E10C947F5AAEE0D8
:10A0E000B0E0E5E7F0E50C94635A1B011E861D867F
:10A0F0009C0140E050E029873A874B875C8700E964
:10A1000011E08D859E858215930509F406C1809125
:10A1100007018093840060E271EA87E090E029857E
:10A120003A854B855C850E94AA59CA01B90197D727
:10A130004B015C012BEA3AEA4AEA50E40E94E358F8
:10A140006B017C0120E030E040E850E4C501B4013F
:10A150000E94E3582B013C0120E030E040E85FE33F
:10A16000C701B601E2D687FD66C020E03FEF4FE7AA
:10A1700057E4C301B2010E94DF5818160CF047C023
:10A1800020E030E04AE754E4C501B401D2D66D8343
:10A190007E838F83988720E030E04AE755E40E9471
:10A1A000E35869837A838B839C8320E030E040E826
:10A1B0005FE3BBD687FD24C020E03FEF4FE757E4C5
:10A1C00069817A818B819C81FAD718169CF420E0F2
:10A1D00030E040E251E46D817E818F819885F3D734
:10A1E00010D76115710589F0C8010197F1F7615029
:10A1F0007109F7CF69817A818B819C8102D702C076
:10A2000061E070E0CB010197F1F760E015C020E05C
:10A2100030E04FE753E4C701B601D1D718163CF43C
:10A22000C301B201EED6CB010197F1F707C0C70118
:10A23000B601E7D601C061E06A95F1F7109284009B
:10A2400020E030E040E85FE3C701B6016ED687FD4D
:10A250005AC020E03FEF4FE757E4C301B201AFD748
:10A2600018160CF03CC020E030E04AE754E4C50189
:10A27000B4015FD64B015C0120E030E04AE755E4D1
:10A28000A2D76B017C0120E030E040E85FE34DD6CF
:10A2900087FD1EC020E03FEF4FE757E4C701B6013E
:10A2A0008ED718168CF420E030E040E251E4C5016E
:10A2B000B40189D7A6D66115710579F0C801019757
:10A2C000F1F761507109F7CFC701B6019AD602C004
:10A2D00061E070E0CB010197F1F760E015C020E08C
:10A2E00030E04FE753E4C701B60169D718163CF4D4
:10A2F000C301B20186D6CB010197F1F707C0C701B0
:10A30000B6017FD601C061E06A95F1F74D855E85A3
:10A310004F5F5F4F5E874D87F4CE2E96E2E10C943F
:10A320007F5AEBE8F0E0808181628083EAE8F0E028
:10A330008081896080830895FC01818190E0982F5D
:10A3400088272081822B0895FC0123816281862F3A
:10A3500090E0A0E0B0E077276627922B2081622B67
:10A360002181722B0895FC01718360830895FC01A3
:10A370007383628351834083089541E050E064E534
:10A3800078E080913305909134050E9401488091D6
:10A3900054080895A5E3B0E0E0EDF1E50C946D5AA2
:10A3A0007C018B016A01CB01F1DBBE016F5F7F4F46
:10A3B000C801FDDB882381F0B601CE0101960E9421
:10A3C000455B892B91F7C801E1DBBE016F5F7F4FD1
:10A3D000C7010E94A84704C0C801D8DB80E090E014
:10A3E000E596E8E00C94895A80913105882351F173
:10A3F0008091570A80FF11C040E052E064E578E0A8
:10A4000080913305909134050E948A490E94C20DC3
:10A410008091570A8E7F8093570A8091570A81FF57
:10A4200011C040E052E065EB7CE0809133059091F3
:10A4300034050E948A490E94C20D8091570A8D7F7F
:10A440008093570A089588E59AE008958AEC97E08A
:10A450000895BC0184ED97E00C944E5B0895BC0117
:10A4600084ED97E00C940F5B089584ED97E00895D8
:10A47000CF93DF93EC0184ED97E00E94695B82301B
:10A4800038F0FC01FF27EC52F84F8FE280831182F5
:10A49000BE0184ED97E00E942F5BDF91CF9108957C
:10A4A00084ED97E00E94695B813081F0815020E06B
:10A4B00030E0E82FE21BF0E02F5F3F4FEC52F84F07
:10A4C00090819F32B1F7108281E0089580E0089575
:10A4D00080913B05882349F180913505909136059F
:10A4E000009729F04DDB10923605109235058091CA
:10A4F000370590913805009731F00E94A2471092DD
:10A500003805109237058091390590913A050097EA
:10A5100031F00E946A0C10923A051092390510929F
:10A52000C9071092C80710923B050895E0913305C2
:10A53000F091340563A574A585A596A50895CF93DC
:10A54000DF936091350570913605AC018091370538
:10A55000909138051FDFEC0190933405809333050B
:10A560000E94F14781E0CD2B09F480E0DF91CF918B
:10A570000895E091540AF091550A09950895809143
:10A580003205882309F442C08091C70781113EC07B
:10A590008091570A80FD12C040E052E064E578E007
:10A5A00080913305909134050E9401482091570A0B
:10A5B00021602093570A81159240B0F08091570A8C
:10A5C00081FD24C040E052E065EB7CE080913305E2
:10A5D000909134050E9401482091570A22602093EF
:10A5E000570A8115924090F481E08093C7078091CB
:10A5F000C8079091C907892B49F0E091C807F091ED
:10A60000C90709951092C9071092C8070895E091EB
:10A61000B30CF091B40C099508950E94C20DE4DECC
:10A6200080913105882309F44BC08091B30C90913F
:10A63000B40C8855974021F44091560A50E016C05A
:10A640008091B30C9091B40C8B56974021F44091BB
:10A65000560A50E019C08091B30C9091B40C8E57FB
:10A66000974039F44091560A50E0539564E578E0FC
:10A670000DC08091B30C9091B40C8659974071F441
:10A680004091560A50E0539565EB7CE0809133058C
:10A69000909134050E948A498091560A0E94C20D09
:10A6A0001092570A1092560A88E197E09093550A43
:10A6B0008093540A8EEA97E09093B40C8093B30C85
:10A6C0000895ABDF8091330590913405009731F008
:10A6D0000E94F14710923405109233051092320512
:10A6E00010923105089599DF8091330590913405DA
:10A6F000FC0147A950AD61AD72AD0E947B4BE0916A
:10A700003305F091340567A970AD81AD92AD089520
:10A71000E0913305F091340547A950AD61AD72ADBC
:10A72000FC0140835183628373830895A4E0B0E009
:10A73000EBE9F3E5D8C669837A838B839C8340E099
:10A74000BE016F5F7F4F80913305909134057BD9B7
:10A7500091E0811101C090E02091540A3091550A96
:10A760002D5B314561F01092570A28E137E03093B4
:10A77000550A2093540A1092560A1092C707892F3F
:10A780002496E2E0CCC6A4E0B0E0E8ECF3E5ABC68A
:10A790009B01AC0188279927DC01821B930BA40B3A
:10A7A000B50B89839A83AB83BC8342E0BE016F5FA4
:10A7B0007F4F809133059091340545D991E0811107
:10A7C00001C090E02091540A3091550A2D5B31452B
:10A7D00061F01092570A28E137E03093550A209330
:10A7E000540A1092560A1092C707892F2496E2E065
:10A7F00096C6C5DEF9CD0895CF92DF92EF92FF9213
:10A80000CF93DF93CDB7DEB7E5970FB6F894DEBFF1
:10A810000FBECDBFC12CD12C7601BE016F5F7F4F23
:10A820008091350590913605C2D9882349F08981F8
:10A830008E3299F38FEFC81AD80AE80AF80AEDCFDA
:10A840008091350590913605A1D9C701B601E596ED
:10A850000FB6F894DEBF0FBECDBFDF91CF91FF9052
:10A86000EF90DF90CF9008950F930E942C0F91E00E
:10A87000811101C090E090933B05992309F468C0D1
:10A8800000E022E631E140E650E160EF7FE08EEE4D
:10A890009DE00E94F10B90933A0580933905892B36
:10A8A00079F40FEF22E631E140E650E160EF7FE01E
:10A8B0008EEE9DE00E94F10B90933A05809339054E
:10A8C0008091390590913A05009709F441C00E94A2
:10A8D0006E4590933805809337050097C9F14EE790
:10A8E0005CE064ED77E060DA81110EC08FE2809366
:10A8F000D4071092D5074EE75CE064ED77E08091D5
:10A9000037059091380550DA6EE77CE08091370585
:10A9100090913805FCD89093360580933505892BA6
:10A92000B9F06ADF6093CC077093CD078093CE07B0
:10A930009093CF071092D0071092D1071092D207B0
:10A940001092D3071092CB071092CA0781E001C082
:10A9500080E00F910895CF93DF93EC0180913B0548
:10A96000811101C081DF6091350570913605AE011E
:10A9700080913705909138050DDD909334058093D3
:10A980003305892BD1F01092570A1092C70788E13E
:10A9900097E09093550A8093540A1092560A81E0EA
:10A9A0008093320510923105109233011092C9073D
:10A9B0001092C807E4DD81E001C080E0DF91CF9113
:10A9C0000895A9E3B0E0E6EEF4E58BC58C01AE0195
:10A9D0004F5F5F4FBC01809135059091360554DA89
:10A9E000811102C010E027C00E94C20DC801B3DF70
:10A9F000182F8823B9F31EAA1FAA18AE19AE40E07B
:10AA0000BE016A5C7F4F80913305909134051BD85D
:10AA1000882341F30E94C20D1092570A2EEA37E0B4
:10AA20003093B40C2093B30C1092560A1092320556
:10AA300081E080933105812FE996E4E06EC5A5E3BE
:10AA4000B0E0E4E2F5E545C56B017C0180913B0592
:10AA5000811101C009DF8091D0079091D107A091A9
:10AA6000D207B091D307C816D906EA06FB0639F417
:10AA7000C114D104E104F10409F0F9C00AC0C816F8
:10AA8000D906EA06FB0628F0C114D104E104F1045A
:10AA900039F5809135059091360578D8812C912C27
:10AAA00054018C149D04AE04BF0408F050C0BE01D4
:10AAB0006F5F7F4F809135059091360578D8882358
:10AAC00009F440C089818E3229F421E0821A91086C
:10AAD000A108B1086FEF861A960AA60AB60AE1CF56
:10AAE0008C159D05AE05BF05B0F52091CA073091C4
:10AAF000CB074C015D01820E931EA11CB11CC81432
:10AB0000D904EA04FB0408F46DC00DC089818E32BB
:10AB100029F421E0821A9108A108B1086FEF861A82
:10AB2000960AA60AB60A8C149D04AE04BF0478F4F3
:10AB3000BE016F5F7F4F809135059091360537D804
:10AB40008111E4CF1092CB071092CA0790C01092E7
:10AB5000CB071092CA0700E010E0C092D007D09255
:10AB6000D107E092D207F092D3078EE3F82EBE0110
:10AB70006F5F7F4F809135059091360518D88823F7
:10AB800009F475C089818E3291F3CE010196A1D569
:10AB9000E82E89A184FF06C0F801E85AF54FF0823B
:10ABA0000F5F1F4FBE016F5F7F4FC801885A954FDF
:10ABB00075D5C8018E0D911D8C010F5F1F4FFC01D3
:10ABC000E85AF54F10822091CA073091CB072F5FCA
:10ABD0003F4F3093CB072093CA078396853292402C
:10ABE00030F245C04C015D0140E050E04F5F5F4FE7
:10ABF000FA01E95AF54F60816111F8CF6FEF861ABB
:10AC0000960AA60AB60A8C149D04AE04BF0471F716
:10AC100046015701881A990AAA0ABB0A2819390954
:10AC200080E090E000E010E082179307D9F0401B2D
:10AC3000510BDA01A85AB54FBA01600F711FFD011F
:10AC4000E00FF11FB080F801E85AF54F0F5F1F4F7A
:10AC5000BB2011F0B082F0CFAB014F5F5F4F10828D
:10AC60000196E2CF9093CB078093CA0776CFE59603
:10AC7000ECE04BC4A5E3B0E0EFE3F6E52CC45C01E7
:10AC800080913505909136050E94C64DC12CD12C7E
:10AC90007601BE016F5F7F4F80913505909136053B
:10ACA0000E94D74D0091350510913605811114C0D1
:10ACB000C8010E94C64D1092D0071092D107109281
:10ACC000D2071092D3071092CB071092CA076FEFEA
:10ACD0007FEF8FEF9FEF22C089818E32D1F2BE01CC
:10ACE0006F5F7F4FC501D1D4892B91F4C8010E94B9
:10ACF000C64D1092D0071092D1071092D207109231
:10AD0000D3071092CB071092CA07B601C70106C03D
:10AD10008FEFC81AD80AE80AF80ABBCFE596EAE02E
:10AD2000F6C3809133059091340502960895A8E00A
:10AD3000B0E0ECE9F6E5D5C380913B058111C8DBB5
:10AD400093DD882309F451C084E598E00E94E11165
:10AD500011E0811101C010E0809137059091380514
:10AD6000E9D804E102D42D833E834F835887809134
:10AD70003705909138050CD9F8D329833A834B8352
:10AD80005C8344E050E0BE016B5F7F4F85EB9CE04D
:10AD900056D444E050E0BE016F5F7F4F89EB9CE0EA
:10ADA0004ED46091370570913805685E7F4F42E060
:10ADB00050E08DEB9CE043D46091370570913805ED
:10ADC0006A5E7F4F42E050E08FEB9CE038D4E09128
:10ADD0003705F091380560817181685F7F4F41E0F0
:10ADE00050E081EC9CE02BD401C010E071DB812F9E
:10ADF0002896E4E092C384E598E00895A4E0B0E0EA
:10AE0000E3E0F7E570C344E050E069EB7CE0CE019D
:10AE1000019615D469817A818B819C812496E2E028
:10AE20007EC3A4E0B0E0E6E1F7E55DC344E050E0B6
:10AE300065EB7CE0CE01019602D469817A818B8139
:10AE40009C812496E2E06BC39ADB93CB0895109229
:10AE5000300510922F0510922E050895809130052F
:10AE6000089580912E0590912F05089581E080939B
:10AE70003301089581E02091330530913405232B6F
:10AE800009F480E008951092570A8EEA97E09093B3
:10AE9000B40C8093B30C1092560A1092320581E0E4
:10AEA0008093310508951092570A88E197E09093B6
:10AEB000550A8093540A1092560A81E08093320515
:10AEC000109231050895A2E0B0E0E8E6F7E50BC383
:10AED00042E050E06DEB7CE0CE010196B0D3898179
:10AEE0009A812296E2E01BC3A2E0B0E0E9E7F7E531
:10AEF000FAC242E050E06FEB7CE0CE0101969FD3B6
:10AF000089819A812296E2E00AC3A1E0B0E0EAE8F2
:10AF1000F7E5E9C241E050E061EC7CE0CE0101964A
:10AF20008ED389812196E2E0FAC2D4D008F481E080
:10AF300008950CD00AC102D140F0F9D030F021F4CC
:10AF40005F3F19F0EBC0511134C1EEC00FD198F33F
:10AF50009923C9F35523B1F3951B550BBB27AA279A
:10AF600062177307840738F09F5F5F4F220F331F0C
:10AF7000441FAA1FA9F333D00E2E3AF0E0E830D0D8
:10AF800091505040E695001CCAF729D0FE2F27D0DB
:10AF9000660F771F881FBB1F261737074807AB07A9
:10AFA000B0E809F0BB0B802DBF01FF2793585F4F1E
:10AFB0002AF09E3F510568F0B1C0FBC05F3FECF343
:10AFC000983EDCF3869577956795B795F7959F5FE3
:10AFD000C9F7880F911D9695879597F90895E1E037
:10AFE000660F771F881FBB1F621773078407BA0796
:10AFF00020F0621B730B840BBA0BEE1F88F7E095F1
:10B000000895BCD088F09F5790F0B92F9927B75179
:10B01000A0F0D1F0660F771F881F991F1AF0BA951C
:10B02000C9F712C0B13081F0C3D0B1E00895C0C0FB
:10B03000672F782F8827B85F39F0B93FCCF3869512
:10B0400077956795B395D9F73EF49095809570956F
:10B0500061957F4F8F4F9F4F0895E89409C097FBEC
:10B060003EF490958095709561957F4F8F4F9F4FDF
:10B070009923A9F0F92F96E9BB279395F695879523
:10B0800077956795B795F111F8CFFAF4BB0F11F4E6
:10B0900060FF1BC06F5F7F4F8F4F9F4F16C088238D
:10B0A00011F096E911C0772321F09EE8872F762FC3
:10B0B00005C0662371F096E8862F70E060E02AF004
:10B0C0009A95660F771F881FDAF7880F96958795F0
:10B0D00097F90895990F0008550FAA0BE0E8FEEFC5
:10B0E00016161706E807F907C0F012161306E4074C
:10B0F000F50798F0621B730B840B950B39F40A2645
:10B1000061F0232B242B252B21F408950A2609F422
:10B11000A140A6958FEF811D811D089597F99F6726
:10B1200080E870E060E008959FEF80EC08950024CF
:10B130000A941616170618060906089500240A949C
:10B1400012161306140605060895092E0394000C22
:10B1500011F4882352F0BB0F40F4BF2B11F460FFB1
:10B1600004C06F5F7F4F8F4F9F4F089557FD9058DA
:10B17000440F551F59F05F3F71F04795880F97FBBB
:10B18000991F61F09F3F79F0879508951216130675
:10B190001406551FF2CF4695F1DF08C016161706A4
:10B1A0001806991FF1CF86957105610508940895D9
:10B1B000E894BB2766277727CB0197F908958ADFA4
:10B1C00008F48FEF08950BD0C0CFB1DF28F0B6DFC1
:10B1D00018F0952309F0A2CFA7CF1124EACFC6DF3C
:10B1E000A0F3959FD1F3950F50E0551F629FF0019A
:10B1F000729FBB27F00DB11D639FAA27F00DB11DF3
:10B20000AA1F649F6627B00DA11D661F829F22277B
:10B21000B00DA11D621F739FB00DA11D621F839F02
:10B22000A00D611D221F749F3327A00D611D231FD8
:10B23000849F600D211D822F762F6A2F11249F5726
:10B2400050408AF0E1F088234AF0EE0FFF1FBB1F49
:10B25000661F771F881F91505040A9F79E3F5105E8
:10B2600070F05CCFA6CF5F3FECF3983EDCF38695A1
:10B2700077956795B795F795E7959F5FC1F7FE2B93
:10B28000880F911D9695879597F90895DB018F9307
:10B290009F9391D0BF91AF91A29F800D911DA39FCD
:10B2A000900DB29F900D11240895991B79E004C070
:10B2B000991F961708F0961B881F7A95C9F78095F5
:10B2C0000895AA1BBB1B51E107C0AA1FBB1FA617ED
:10B2D000B70710F0A61BB70B881F991F5A95A9F73F
:10B2E00080959095BC01CD01089597FB072E16F42B
:10B2F000009406D077FD08D0E4DF07FC05D03EF4CB
:10B30000909581959F4F0895709561957F4F089511
:10B31000A1E21A2EAA1BBB1BFD010DC0AA1FBB1F59
:10B32000EE1FFF1FA217B307E407F50720F0A21BCB
:10B33000B30BE40BF50B661F771F881F991F1A9438
:10B3400069F760957095809590959B01AC01BD0162
:10B35000CF010895052E97FB16F400940FD057FDEA
:10B3600005D0D6DF07FC02D046F408C050954095C2
:10B37000309521953F4F4F4F5F4F089590958095A1
:10B38000709561957F4F8F4F9F4F0895EE0FFF1F70
:10B390000590F491E02D0994A29FB001B39FC001E4
:10B3A000A39F700D811D1124911DB29F700D811DF1
:10B3B0001124911D0895F0DFA59F900DB49F900D6D
:10B3C000A49F800D911D11240895B7FFF4CFF3DFE2
:10B3D000821B930B0895DF93CF931F930F939A9D36
:10B3E000F02D219FF00D8B9DF00D8A9DE02DF10D2C
:10B3F000039FF00D029FE00DF11D4E9DE00DF11D2C
:10B400005E9DF00D4F9DF00D7F936F93BF92AF92B5
:10B410005F934F93D501C0DF8B01AC01D701BCDF37
:10B42000EB01E80FF91FD6011FD02F913F91D601F4
:10B43000B3DFC60FD71FE81FF91FAF91BF9114D01C
:10B440002F913F91A9DFC60FD71FE81FF91FD60123
:10B45000A3DFE60FF71F9801BE01CF0111240F9162
:10B460001F91CF91DF91089597DF460F571FC81F97
:10B47000D91F08F431960895E894DF93CF93FC0127
:10B48000DB018ADF7F936F93E9019A01AC01BF93DF
:10B49000AF933F932F93DF017FDF26F46C1B7D0B6F
:10B4A000820B930B9E01EB01FC01DEDFAF91BF919C
:10B4B0002F913F91D9DFBE01CF01F9012F913F912B
:10B4C000CF91DF9108952F923F924F925F926F92AA
:10B4D0007F928F929F92AF92BF92CF92DF92EF9224
:10B4E000FF920F931F93CF93DF93CDB7DEB7CA1BA5
:10B4F000DB0B0FB6F894DEBF0FBECDBF09942A88D0
:10B50000398848885F846E847D848C849B84AA8477
:10B51000B984C884DF80EE80FD800C811B81AA8104
:10B52000B981CE0FD11D0FB6F894DEBF0FBECDBFCF
:10B53000ED0108950F93083090F0982F872F762F04
:10B54000652F542F432F322F22270850F4CF220F7C
:10B55000331F441F551F661F771F881F991F0A95A9
:10B56000B2F70F91089597FB10F8169400080F9307
:10B57000083098F00850232F342F452F562F672F6F
:10B58000782F892F902DF4CF0594979587957795EF
:10B59000679557954795379527950A95AAF70F917F
:10B5A00008952A0D3B1D4C1D5D1D6E1D7F1D801FC6
:10B5B000911F08950024A7FD00942A0F301D401DFF
:10B5C000501D601D701D801D901D08952A193B0996
:10B5D0004C095D096E097F09800B910B08952A15AE
:10B5E0003B054C055D056E057F05800791070895B5
:10B5F0000024A7FD00942A1730054005500560057A
:10B600007005800590050895FB01DC010D90002078
:10B61000E9F7119705900D920020E1F70895FB01DD
:10B62000DC0105900D920020E1F70895FC010590E2
:10B630000020E9F7809590958E0F9F1F0895FB01DC
:10B64000DC0102C001900D9241505040D8F708959E
:10B65000DC0101C06D9341505040E0F70895FB01BB
:10B66000DC010D900020E9F7119701900D92002068
:10B67000E1F70895FC018191861721F08823D9F71D
:10B68000992708953197CF010895FB01DC018D9131
:10B69000019080190110D9F3990B0895FB01DC0189
:10B6A00001900D920020E1F70895DC01FB0141506B
:10B6B000504058F049F001900D920020C1F7E61B70
:10B6C000F70B3197CF0108951C9201900020E9F704
:10B6D000F6CFFC0101900020E9F7809590958E0F40
:10B6E0009F1F0895FB01DC014150504030F08D91C7
:10B6F0000190801919F40020B9F7881B990B08955F
:10B70000FB01DC014150504048F001900D920020B7
:10B71000C9F701C01D9241505040E0F70895FC0167
:10B7200081E090E00190061609F4CF010020D1F7E6
:10B7300001970895BB274A3031F4992322F4BDE2E2
:10B74000909581959F4F30C0BB272A3051F49923A3
:10B7500042F4BDE290958095709561957F4F8F4F33
:10B760009F4F01C0BB27FA01A62F62177105810503
:10B770009105330B30FB66F0AA27660F771F881FF1
:10B78000991FAA1FA21710F0A21B63953850A9F7A2
:10B79000A05DAA3308F0A95DA19336F7B111B1936A
:10B7A0001082CA018CC2BB27FB015527AA27880F2C
:10B7B000991FAA1FA41710F0A41B83955051B9F725
:10B7C000A05DAA3308F0A95DA193009779F7B111A4
:10B7D000B1931192CB0173C20F931F93CF93DF9359
:10B7E000CDB7DEB72E970FB6F894DEBF0FBECDBF34
:10B7F0000D891E898EE08C831A8309838FEF9FE762
:10B800009E838D83AE01475E5F4F6F89788DCE0139
:10B81000019610D0EF81F885E00FF11F10822E966F
:10B820000FB6F894DEBF0FBECDBFDF91CF911F9151
:10B830000F9108952F923F924F925F926F927F9255
:10B840008F929F92AF92BF92CF92DF92EF92FF9230
:10B850000F931F93CF93DF93CDB7DEB72C970FB61F
:10B86000F894DEBF0FBECDBF7C016B018A01FC01E5
:10B8700017821682838181FFB0C1CE0101964C01EF
:10B88000F7019381F60193FD859193FF81916F01FB
:10B89000882309F49EC1853239F493FD859193FF85
:10B8A00081916F01853221F4B70190E018D2E8CF81
:10B8B000512C312C20E02032A0F48B3269F030F48E
:10B8C000803259F0833269F420612CC08D3239F016
:10B8D000803339F4216026C02260246023C02860B0
:10B8E00021C027FD27C030ED380F3A3078F426FF0D
:10B8F00006C0FAE05F9E300D1124532E13C08AE07B
:10B90000389E300D1124332E20620CC08E3221F46B
:10B9100026FD5FC1206406C08C3611F4206802C089
:10B92000883641F4F60193FD859193FF81916F0173
:10B930008111C1CF982F9F7D9554933028F40C5FCF
:10B940001F4FFFE3F9830DC0833631F0833771F069
:10B95000833509F057C021C0F801808189830E5FCB
:10B960001F4F44244394512C540114C03801F2E079
:10B970006F0E711CF801A080B18026FF03C0652DF9
:10B9800070E002C06FEF7FEFC5012C878DD12C01D5
:10B9900083012C852F77222E16C03801F2E06F0E1E
:10B9A000711CF801A080B18026FF03C0652D70E0F6
:10B9B00002C06FEF7FEFC5012C876BD12C012C8566
:10B9C0002068222E830123FC19C0832D90E04816A5
:10B9D0005906A0F4B70180E290E081D13A94F5CF06
:10B9E000F50127FC859127FE81915F01B70190E069
:10B9F00076D131103A94F1E04F1A510841145104B4
:10BA000079F7DEC0843611F0893631F5F80127FF69
:10BA100007C060817181828193810C5F1F4F08C0D4
:10BA200060817181882777FD8095982F0E5F1F4F69
:10BA30002F76B22E97FF09C09095809570956195ED
:10BA40007F4F8F4F9F4F2068B22E2AE030E0A40135
:10BA500078D1A82EA81843C0853729F42F7EB22E9E
:10BA60002AE030E025C0F22FF97FBF2E8F36C1F0DB
:10BA700018F4883579F0ADC0803719F0883721F097
:10BA8000A8C02F2F2061B22EB4FE0DC08B2D846074
:10BA9000B82E09C024FF0AC09F2F9660B92E06C099
:10BAA00028E030E005C020E130E002C020E132E0D3
:10BAB000F801B7FE07C060817181828193810C5FBC
:10BAC0001F4F06C06081718180E090E00E5F1F4FC4
:10BAD000A40137D1A82EA818FB2DFF77BF2EB6FEE4
:10BAE0000BC02B2D2E7FA51450F4B4FE0AC0B2FC5F
:10BAF00008C02B2D2E7E05C07A2C2B2D03C07A2C4E
:10BB000001C0752C24FF0DC0FE01EA0DF11D8081DE
:10BB1000803311F4297E09C022FF06C07394739408
:10BB200004C0822F867809F0739423FD12C020FF91
:10BB300006C05A2C731418F4530C5718732C731432
:10BB400060F4B70180E290E02C87C9D073942C8513
:10BB5000F6CF731410F4371801C0312C24FF11C034
:10BB6000B70180E390E02C87BAD02C8522FF16C065
:10BB700021FF03C088E590E002C088E790E0B701AC
:10BB80000CC0822F867851F021FD02C080E201C0F6
:10BB90008BE227FD8DE2B70190E0A1D0A51430F42F
:10BBA000B70180E390E09BD05A94F8CFAA94F401B7
:10BBB000EA0DF11D8081B70190E091D0A110F6CF80
:10BBC000332009F45DCEB70180E290E088D03A944A
:10BBD000F7CFF7018681978102C08FEF9FEF2C96F8
:10BBE0000FB6F894DEBF0FBECDBFDF91CF911F918E
:10BBF0000F91FF90EF90DF90CF90BF90AF909F900C
:10BC00008F907F906F905F904F903F902F9008950E
:10BC1000DC01CB01FC01E199FECF06C0FFBBEEBB0E
:10BC2000E09A31960DB20D9241505040B8F7089508
:10BC3000E199FECF9FBB8EBBE09A99278DB3089503
:10BC4000A8E1B0E042E050E0E5CFDC01A40FB51F71
:10BC50004150504040F0CB01840F951F2E9105D0EC
:10BC600041505040D8F70895262FE199FECF9FBB51
:10BC70008EBBE09A01970DB2021631F02DBB0FB6C4
:10BC8000F894E29AE19A0FBE08950196272FEDDF0E
:10BC9000EBCFFC010590615070400110D8F7809502
:10BCA00090958E0F9F1F0895FC0161507040019088
:10BCB0000110D8F7809590958E0F9F1F0895DC0195
:10BCC000FC01672F71917723E1F7329704C07C91D3
:10BCD0006D9370836291AE17BF07C8F308950F93F9
:10BCE0001F93CF93DF93182F092FEB018B8181FDD9
:10BCF00003C08FEF9FEF20C082FF10C04E815F8195
:10BD00002C813D81421753077CF4E881F9819F0122
:10BD10002F5F3F4F39832883108306C0E885F9855C
:10BD2000812F0995892B29F72E813F812F5F3F4F66
:10BD30003F832E83812F902FDF91CF911F910F9101
:10BD40000895FA01AA27283051F1203181F1E894B1
:10BD50006F936E7F6E5F7F4F8F4F9F4FAF4FB1E0FE
:10BD60003ED0B4E03CD0670F781F891F9A1FA11DF9
:10BD7000680F791F8A1F911DA11D6A0F711D811DFA
:10BD8000911DA11D20D009F468943F912AE0269FBF
:10BD900011243019305D3193DEF6CF010895462F1E
:10BDA0004770405D4193B3E00FD0C9F7F6CF462FFF
:10BDB0004F70405D4A3318F0495D31FD4052419368
:10BDC00002D0A9F7EACFB4E0A69597958795779525
:10BDD0006795BA95C9F700976105710508959B01AC
:10BDE000AC010A2E06945795479537952795BA9535
:10BDF000C9F7620F731F841F951FA01D0895F89443
:02BE0000FFCF72
:10BE0200010000000422568001030507090E1012EA
:0EBE12001416181C1E2F007706740671060009
:00000001FF
